:100000000C9418040C94E61E0C94BF1E0C9440042F
:100010000C9440040C9440040C9440040C94400450
:100020000C9440040C9440040C9440040C94400440
:100030000C9440040C94651F0C9440040C944004F0
:100040000C94751E0C9440040C94331F0C940D1FDB
:100050000C9440040C9440040C9440040C94400410
:100060000C948C1F0C94400407634236B79BD8A7AE
:100070001A39685618AEBAAB558C1D3CB7CC5763CD
:10008000BD6DEDFD753EF6177231BF000000803F7B
:1000900008000000BE922449123EABAAAA2ABECD97
:1000A000CCCC4C3E00000080BEABAAAAAA3E000009
:1000B0000000BF000000803F000000000008417801
:1000C000D3BB4387D1133D190E3CC3BD4282AD2B38
:1000D0003E68EC8276BED98FE1A93E4C80EFFFBE30
:1000E00001C4FF7F3F000000000001000819130455
:1000F000E81A0010191302E84C0011191301E882E4
:100100000010191301E8B40011191301E8EA0010F6
:10011000191302E81C0110191302E84E01111913FA
:1001200001E8000303070F3FFFFF07070707070763
:1001300007070707070707070707070707E01FF86D
:100140003FFC7C3E700FF00FE007E0070007000760
:10015000000F001E003C00F803F007C01F003C0029
:10016000380070006000E000FFFFFFFFFFFF07F0B6
:1001700007FE07FF8783C380F38039C01CE00E00B1
:1001800007000F007F003F001FE00078001E0007FF
:100190000003F001F800FE00770073E0F8FFF83F7D
:1001A000F807F00000380038007800F800F801F88F
:1001B00003B8033807380E381C3818383838703808
:1001C0006038E038FFFFFFFFFFFF003800380038DD
:1001D0000038003800381FFF0FFF8FFFC700038073
:1001E00001C000E000700039F03FFE1FFF8F83E781
:1001F00000F0003C000E000700038001C000FC007E
:10020000EF0073C0F0FFF83FF807E00003E00FF8DD
:100210001FFC3C1E380E700E70006000E000E3E032
:10022000EFF8FFFCFC3EF00EF00FE007E007E00700
:100230006007700F700E3C3E3FFC1FF807E0FFFFA9
:10024000FFFFFFFF0006000E001C001800380070C2
:10025000006000E000C001C001800380038007004F
:10026000070007000E000E000E000C001C001C0012
:1002700007F00FFE0FFF8783C780F38039C01CE0B3
:100280000E780F1E0F07FF01FF03FFE3E0F9C01D0B
:10029000C00FE003F001F800FC00F70073E0F8FF86
:1002A000F83FF807F000002201EA0031003800387A
:1002B00000000000003E5B4F5B3E3E6B4F6B3E1C00
:1002C0003E7C3E1C183C7E3C181C577D571C1C5E17
:1002D0007F5E1C00183C1800FFE7C3E7FF001824EE
:1002E0001800FFE7DBE7FF30483A060E2629792998
:1002F00026407F050507407F05253F5A3CE73C5ACD
:100300007F3E1C1C08081C1C3E7F14227F22145FA9
:100310005F005F5F06097F017F006689956A606004
:1003200060606094A2FFA29408047E040810207EFE
:10033000201008082A1C08081C2A08081E10101083
:10034000100C1E0C1E0C30383E3830060E3E0E06C9
:10035000000000000000005F00000007000700141C
:100360007F147F14242A7F2A1223130864623649DB
:100370005620500008070300001C224100004122C3
:100380001C002A1C7F1C2A08083E080800807030C8
:100390000008080808080000606000201008040237
:1003A0003E5149453E00427F40007249494946213D
:1003B00041494D331814127F1027454545393C4AB1
:1003C00049493141211109073649494936464949C8
:1003D000291E000014000000403400000008142210
:1003E000411414141414004122140802015909067E
:1003F0003E415D594E7C1211127C7F494949363E7F
:10040000414141227F4141413E7F494949417F0964
:100410000909013E414151737F0808087F00417F6F
:1004200041002040413F017F081422417F4040406D
:10043000407F021C027F7F0408107F3E4141413E05
:100440007F090909063E4151215E7F091929462687
:100450004949493203017F01033F4040403F1F208B
:1004600040201F3F4038403F631408146303047862
:1004700004036159494D43007F4141410204081082
:1004800020004141417F04020102044040404040BD
:10049000000307080020545478407F28444438382B
:1004A00044444428384444287F385454541800089D
:1004B0007E090218A4A49C787F0804047800447D77
:1004C00040002040403D007F1028440000417F4014
:1004D000007C047804787C08040478384444443868
:1004E000FC1824241818242418FC7C080404084848
:1004F0005454542404043F44243C4040207C1C2099
:1005000040201C3C4030403C44281028444C9090F3
:10051000907C4464544C440008364100000077004D
:1005200000004136080002010204023C2623263C5A
:100530001EA1A161123A4040207A385454555921E5
:1005400055557941225454784221555478402054CD
:100550005579400C1E52721239555555593954541B
:10056000545939555454580000457C410002457D8A
:10057000420001457C407D1211127DF0282528F0B3
:100580007C545545002054547C547C0A097F4932E0
:10059000494949323A4444443A324A4848303A4157
:1005A00041217A3A42402078009DA0A07D3D424200
:1005B000423D3D4040403D3C24FF2424487E494389
:1005C000662B2FFC2F2BFF0929F620C0887E0903FC
:1005D00020545479410000447D413048484A323823
:1005E0004040227A007A0A0A727D0D19317D26294F
:1005F000292F28262929292630484D402038080847
:10060000080808080808382F10C8ACBA2F1028347A
:10061000FA00007B000008142A142222142A14086D
:100620005500550055AA55AA55AAFF55FF55FF007C
:100630000000FF00101010FF00141414FF00101031
:10064000FF00FF1010F010F0141414FC001414F745
:1006500000FF0000FF00FF1414F404FC1414171032
:100660001F10101F101F1414141F00101010F00082
:100670000000001F101010101F10101010F01000BC
:100680000000FF101010101010101010FF100000CC
:1006900000FF140000FF00FF00001F10170000FC07
:1006A00004F414141710171414F404F40000FF00D9
:1006B000F714141414141414F700F7141414171462
:1006C00010101F101F141414F4141010F010F00068
:1006D000001F101F0000001F14000000FC14000089
:1006E000F010F01010FF10FF141414FF141010106D
:1006F0001F00000000F010FFFFFFFFFFF0F0F0F020
:10070000F0FFFFFF0000000000FFFF0F0F0F0F0FB3
:100710003844443844FC4A4A4A347E0202060602FF
:100720007E027E0263554941633844443C04407E66
:10073000201E2006027E020299A5E7A5991C2A49DF
:100740002A1C4C7201724C304A4D4D30304878486A
:1007500030BC625A463D3E494949007E0101017E56
:100760002A2A2A2A2A44445F444440514A444040A9
:10077000444A51400000FF0103E080FF00000808E8
:100780006B6B083612362436060F090F0600001868
:10079000180000001010003040FF0101001F01018F
:1007A0001E00191D1712003C3C3C3C0000000000DC
:1007B0000901809611800A3A81550A3601082A04F7
:1007C000000000F02B040000014021800A13800A81
:1007D00029800A00000000240027002A00000000F1
:1007E000002300260029000000000800020100008C
:1007F00003040700000000000000000102040810CC
:10080000204080010204081020010204081020008A
:10081000000000250028002B000404040404040444
:100820000402020202020203030303030300A720DF
:1008300011241FBECFEFD8E0DEBFCDBF12E0A0E095
:10084000B1E0EEE9FCE602C005900D92A23FB107CF
:10085000D9F724E0A2EFB2E001C01D92AF3FB2078A
:10086000E1F714E0C8E1D4E004C02197FE010E9442
:100870001D35C731D107C9F70E94AE210C944D3602
:100880000C940000FC01538D448D252F30E0842F03
:1008900090E0821B930B541710F0CF9608950197A8
:1008A0000895FC01918D828D981761F0A28DAE0F95
:1008B000BF2FB11D5D968C91928D9F5F9F73928F1C
:1008C00090E008958FEF9FEF0895FC01918D828D48
:1008D000981731F0828DE80FF11D858D90E0089515
:1008E0008FEF9FEF0895FC01918D228D892F90E06D
:1008F000805C9F4F821B91098F7399270895FC019B
:10090000A48DA80FB92FB11DA35ABF4F2C91848D70
:1009100090E001968F739927848FA689B7892C93CD
:10092000A089B1898C91837080648C93938D848D20
:10093000981306C00288F389E02D80818F7D808323
:100940000895EF92FF920F931F93CF93DF93EC01E3
:1009500081E0888F9B8D8C8D98131AC0E889F98966
:10096000808185FF15C09FB7F894EE89FF89608369
:10097000E889F98980818370806480839FBF81E0EA
:1009800090E0DF91CF911F910F91FF90EF9008952C
:10099000F62E0B8D10E00F5F1F4F0F731127E02E07
:1009A0008C8D8E110CC00FB607FCFACFE889F9893F
:1009B000808185FFF5CFCE010E947F04F1CFEB8DC2
:1009C000EC0FFD2FF11DE35AFF4FF0829FB7F89413
:1009D0000B8FEA89FB8980818062CFCFCF93DF9331
:1009E000EC01888D8823B9F0AA89BB89E889F98947
:1009F0008C9185FD03C0808186FD0DC00FB607FC7C
:100A0000F7CF8C9185FFF2CF808185FFEDCFCE01AE
:100A10000E947F04E9CFDF91CF91089585EF93E0A5
:100A20000E94730421E0892B09F420E0822F0895AD
:100A300080E090E0892B29F00E940E0581110C9432
:100A400000000895833081F028F4813099F08230DD
:100A5000A9F008958730A9F08830C9F08430B1F446
:100A6000809180008F7D03C0809180008F7780937C
:100A70008000089584B58F7784BD089584B58F7DF7
:100A8000FBCF8091B0008F778093B0000895809164
:100A9000B0008F7DF9CFCF93DF93282F30E0F9019D
:100AA000E951F84F8491F901E550F84FD491F901DB
:100AB000E75EF74FC491CC23A1F081110E9422057B
:100AC000EC2FF0E0EE0FFF1FE352F84FA591B49129
:100AD000EC91ED2381E090E009F480E0DF91CF918B
:100AE000089580E090E0FACF1F93CF93DF93282FF3
:100AF00030E0F901E951F84F8491F901E550F84FE0
:100B0000D491F901E75EF74FC491CC23A9F0162FD9
:100B100081110E942205EC2FF0E0EE0FFF1FE15F34
:100B2000F74FA591B4918FB7F894EC91111108C0CB
:100B3000D095DE23DC938FBFDF91CF911F91089575
:100B4000DE2BF8CFCF93DF9390E0FC01E550F84F18
:100B50002491875E974FFC0184918823C9F090E02F
:100B6000880F991FFC01ED52F84FA591B491FC013B
:100B7000E15FF74FC591D49161110DC09FB7F89413
:100B80008C91209582238C938881282328839FBF72
:100B9000DF91CF910895623051F49FB7F8943C9162
:100BA000822F809583238C93E8812E2BEFCF8FB7F4
:100BB000F894EC912E2B2C938FBFEACF8E3008F057
:100BC0008E508770806480937C0080917A0080646E
:100BD00080937A0080917A0086FDFCCF8091780026
:100BE0009091790008953FB7F8948091EA0390912D
:100BF000EB03A091EC03B091ED0326B5A89B05C0D3
:100C00002F3F19F00196A11DB11D3FBFBA2FA92F8B
:100C1000982F8827BC01CD01620F711D811D911D88
:100C200042E0660F771F881F991F4A95D1F70895F4
:100C30008F929F92AF92BF92CF92DF92EF92FF92EC
:100C40006B017C010E94F3054B015C01C114D104CE
:100C5000E104F104B9F00E94F305681979098A09E1
:100C60009B09683E73408105910580F321E0C21A1B
:100C7000D108E108F10888EE880E83E0981EA11CD7
:100C8000B11CE4CFFF90EF90DF90CF90BF90AF907A
:100C90009F908F9008952FB7F8946091E60370911C
:100CA000E7038091E8039091E9032FBF0895089529
:100CB000AF92BF92CF92DF92EF92FF920F931F936A
:100CC000CF93DF936C017B018B01040F151FEB01A8
:100CD0005E01AE18BF08C017D10759F06991D6015F
:100CE000ED91FC910190F081E02DC6010995892BD1
:100CF00079F7C501DF91CF911F910F91FF90EF9090
:100D0000DF90CF90BF90AF9008950895FC0190853B
:100D1000957081E0953009F080E00895CF92DF92E0
:100D2000EF92FF920F931F93CF93DF93EC0188858F
:100D30008B7F8887E881F9810190F081E02DCE01D9
:100D40000995182F8885869581701817B9F00E942B
:100D50004B066A837B838C839D83888592E08927F9
:100D60008887888582FB882780F9DF91CF911F9142
:100D70000F91FF90EF90DF90CF9008950E944B0667
:100D8000CA80DB80EC80FD80AB01BC014C195D09A1
:100D90006E097F098E819F81B0E0A0E04817590756
:100DA0006A077B07F0F2888581701817D1F20E94DC
:100DB0004B066A837B838C839D83888591E089279A
:100DC000846088870E944B0609851A852B853C859F
:100DD000601B710B820B930B6D877E878F87988BBF
:100DE0000E944B0669877A878B879C87BACFCF93FF
:100DF000DF93EC011886E881F9810190F081E02D04
:100E00000995882319F08885836088870E944B069E
:100E10006A837B838C839D83DF91CF910895862F96
:100E2000642F0C94A205FC0181890E944B0521E0EE
:100E3000892B09F420E0822F089520912803260FA2
:100E40003327331F21323105ECF420914C03FC0190
:100E500090E080E0243069F082E00895A0912803BA
:100E60002191AC01485F5C4FA40FB52FB11D2C93AD
:100E70000196861798F380912803680F60932803E2
:100E800080E0089581E0089508958FEF9FEF089521
:100E90008FEF9FEF08958091010390E091958195E8
:100EA00091090895CF93DF93CB01EA01642F0E944B
:100EB0001D07CE01DF91CF910895CF93DF931F924D
:100EC000CDB7DEB7698361E0CE0101960E941D07B0
:100ED00081E090E00F90DF91CF910895FC01A5A1F2
:100EE000B6A18C9192A589238C93A5A1B6A18C91D2
:100EF00091A5892B8C930895DC019396ED91FC913B
:100F00009497908198968C91892380830895DC0131
:100F10009396ED91FC919497908197968C91892B63
:100F200080830895DC019196ED91FC9192979081D8
:100F300096968C91892380830895DC019196ED919A
:100F4000FC919297908195968C91892B808308953E
:100F5000CF92DF92EF92FF921F93CF93DF93EC013A
:100F60006A017B018DA9811123C08F2D9927AA27A2
:100F7000BB278EBD0DB407FEFDCFC701AA27BB2737
:100F80008EBD0DB407FEFDCFBB27AF2D9E2D8D2D41
:100F90008EBD0DB407FEFDCFCEBC0DB407FEFDCF58
:100FA000DF91CF911F91FF90EF90DF90CF90089548
:100FB0008130B1F410E2CE01F7FE0FC00E949D0710
:100FC000CE010E948707CE010E947C07CC0CDD1C5D
:100FD000EE1CFF1C115079F7E3CF0E949207F0CF6F
:100FE000EF8DF8A18F2D9927AA27BB278083CE01EB
:100FF0000E946E07EF8DF8A1C701AA27BB27808347
:10100000CE010E946E07EF8DF8A1BB27AF2D9E2D5C
:101010008D2D8083CE010E946E07EF8DF8A1C082D6
:10102000CE01DF91CF911F91FF90EF90DF90CF9095
:101030000C946E07FF920F931F93CF93DF93EC01F5
:101040008B018DA981110EC01EBD0DB407FEFDCF11
:101050000EBD0DB407FEFDCFDF91CF911F910F9113
:10106000FF9008958130B1F490E1F92ECE0117FF81
:101070000EC00E949D07CE010E948707CE010E94EC
:101080007C07000F111FFA94F110F0CFE5CF0E94FA
:101090009207F1CFEF8DF8A11083CE010E946E0769
:1010A000EF8DF8A10083CE01DF91CF911F910F91B9
:1010B000FF900C946E070F931F93CF93DF93EC0177
:1010C000162F8DA9811109C06EBD0DB407FEFDCF8D
:1010D000DF91CF911F910F910895813099F408E02D
:1010E000CE0117FF0CC00E949D07CE010E9487070A
:1010F000110FCE010E947C07015091F7E9CF0E94A9
:101100009207F3CFEF8DF8A16083CE01DF91CF91ED
:101110001F910F910C946E07CF93DF93EC01ED8D2F
:10112000FE8D80819CA989238083CE010E945B086B
:10113000ED8DFE8D80819BA9892B8083DF91CF91DE
:1011400008958F929F92AF92BF92CF92DF92EF92CB
:10115000FF920F931F93CF93DF93EC0189AD9AAD6C
:10116000680F791F8BAD9CAD480F591F2150310975
:10117000260F371F4901B12CA12CCB01B0E0A0E014
:10118000DC0199278827882A992AAA2ABB2A68017C
:1011900081E0C81AD108C40ED51EF12CE12C70E0F4
:1011A00060E0BA0155274427C42AD52AE62AF72A3F
:1011B0006AE2CE010E948C08B501A401CE010E9412
:1011C000A8076BE2CE010E948C08B701A601CE01F0
:1011D0000E94A8076CE2CE01DF91CF911F910F9181
:1011E000FF90EF90DF90CF90BF90AF909F908F9047
:1011F0000C948C08FC0185A9811104C091A182A1E5
:101200009CBD8DBD08951F93CF93DF93EC01162FE6
:10121000E881F9810284F385E02D0995112371F0AD
:101220006DADCE010E948C08E881F9810688F789AE
:10123000E02DCE01DF91CF911F9109946EADF1CFDA
:10124000AF92BF92CF92DF92EF92FF920F931F93D4
:10125000CF93DF93EC0177FD38C0888599856817B7
:1012600079079CF557FD31C08A859B85481759073A
:1012700064F569017A015B01E881F9810284F385F3
:10128000E02DCE010995E881F98102A4F3A5E02DB6
:1012900001E010E021E030E0A701B501CE010995A1
:1012A000B601CE010E941A08E881F9810688F78903
:1012B000E02DCE01DF91CF911F910F91FF90EF9024
:1012C000DF90CF90BF90AF900994DF91CF911F91A5
:1012D0000F91FF90EF90DF90CF90BF90AF90089567
:1012E0008F929F92AF92BF92CF92DF92EF92FF9236
:1012F0000F931F93CF93DF93EC0149015701E881CE
:10130000F98102A4F3A5E02D09959401D8010E946A
:101310000E356B017C01C114D104E104F10409F420
:101320007DC08DA9811115C081E0C81AD108E108DE
:10133000F1088FEFC816D806E806F80609F46EC063
:10134000BEBC0DB407FEFDCFAEBC0DB407FEFDCF95
:10135000EBCF813099F581E0C81AD108E108F10896
:101360008FEFC816D806E806F80609F457C00B2D0B
:1013700018E0CE0107FF1CC00E949D07CE010E940D
:101380008707CE010E947C07000F115091F70A2DAC
:1013900018E0CE0107FF0FC00E949D07CE010E94FA
:1013A0008707CE010E947C07000F115091F7D3CF21
:1013B0000E949207E3CF0E949207F0CFBA1016C0A6
:1013C000CC0CDD1CEE1CFF1CEF8DF8A1B08281E07F
:1013D000C81AD108E108F1088FEFC816D806E80648
:1013E000F806E1F0CE010E946E07F1CF81E0C81A45
:1013F000D108E108F1088FEFC816D806E806F8060C
:1014000069F0EF8DF8A1B082CE010E946E07EF8DDA
:10141000F8A1A082CE010E946E07E8CFDF91CF91A4
:101420001F910F91FF90EF90DF90CF90BF90AF9002
:101430009F908F9008958F929F92AF92BF92CF927C
:10144000DF92EF92FF920F931F93CF93DF934C01A4
:10145000EB016A01590137FF07C0C9010196C80FA6
:10146000D91FB194A194B108F401A085B185CA1720
:10147000DB070CF058C017FF07C0C8010196C80E63
:10148000D91E119501951109F40182859385C8161D
:10149000D9060CF048C0FE01EA0DFB1DAF0141501A
:1014A000510957FD40C0B601600F711F9B012150CB
:1014B000310937FD38C0D7FF03C05F01D0E0C0E07D
:1014C000D7FE03C08B01D12CC12C4A175B071CF03F
:1014D0005D01AC1ABD0A281739071CF08C010C19E4
:1014E0001D09D401ED91FC910284F385E02DC40126
:1014F00009959501A601BE01C4010E947009D4019D
:10150000ED91FC910688F789E02DC401DF91CF9120
:101510001F910F91FF90EF90DF90CF90BF90AF9011
:101520009F908F900994DF91CF911F910F91FF9021
:10153000EF90DF90CF90BF90AF909F908F900895E5
:10154000EF92FF920F931F932115310529F001159A
:10155000110511F00E941B0A1F910F91FF90EF904F
:1015600008958F929F92AF92BF92CF92DF92EF92A7
:10157000FF920F931F93CF93DF935C014B016A019E
:10158000E90177FD52C0DC0118968D919C91681796
:1015900079070CF04AC0209709F447C037FF07C00D
:1015A000C9010196C80ED91ED195C195D109F50181
:1015B00082859385C816D906C4F5A6014C0F5D1F18
:1015C0009A012150310937FD30C0D7FE03C0EA012E
:1015D000D12CC12C281739071CF0EC01CC19DD09DE
:1015E000D501ED91FC910284F385E02DC5010995AB
:1015F00078018E0121E030E0A601B401C5010E940E
:101600007009D501ED91FC910688F789E02DC5019F
:10161000DF91CF911F910F91FF90EF90DF90CF90CE
:10162000BF90AF909F908F900994DF91CF911F91C1
:101630000F91FF90EF90DF90CF90BF90AF909F9071
:101640008F9008958F929F92AF92BF92CF92DF9228
:10165000EF92FF920F931F93CF93DF935C016B0187
:101660004A01E90157FD52C0DC011A968D919C9107
:10167000481759070CF04AC0209709F447C037FFB4
:1016800007C0C9010196C80ED91ED195C195D109CF
:10169000F50180859185C816D906C4F5A6014C0FC1
:1016A0005D1F9A012150310937FD30C0D7FE03C0BC
:1016B000EA01D12CC12C281739071CF0EC01CC19F8
:1016C000DD09D501ED91FC910284F385E02DC50182
:1016D0000995780101E010E09E01A401B601C50161
:1016E0000E947009D501ED91FC910688F789E02DE3
:1016F000C501DF91CF911F910F91FF90EF90DF9087
:10170000CF90BF90AF909F908F900994DF91CF9131
:101710001F910F91FF90EF90DF90CF90BF90AF900F
:101720009F908F900895EF92FF920F931F93CF9306
:10173000DF9377FD32C0DC011896ED91FC916E17B6
:101740007F075CF52115310541F137FF07C0F9012D
:1017500031964E0F5F1F319521953109DC011A96A4
:10176000ED91FC914E175F07C4F4EA01C20FD31F3D
:10177000DE011197B7FD11C057FF03C09E0150E075
:1017800040E0AE17BF071CF09F01241B350B78010A
:10179000890121E030E00E947009DF91CF911F9113
:1017A0000F91FF90EF900895EF92FF920F931F9388
:1017B000CF93DF9357FD31C0DC011A96ED91FC9178
:1017C0004E175F0754F52115310539F137FF07C072
:1017D000F90131966E0F7F1F319521953109DC019A
:1017E0001896ED91FC916E177F07BCF4EB01C20FC8
:1017F000D31FDE011197B7FD10C077FF03C09E0114
:1018000070E060E0AE17BF071CF09F01261B370B8E
:10181000780101E010E00E947009DF91CF911F91E3
:101820000F91FF90EF9008958F929F92AF92BF9289
:10183000CF92DF92EF92FF920F931F93CF93DF939C
:1018400047012115310509F44BC00115110509F4B3
:1018500047C037FF07C0F90131966E0F7F1F3195E2
:1018600021953109DC011896AD90BC906A157B0575
:10187000BCF517FF07C0F80131964E0F5F1F119599
:1018800001951109DC011A96ED91FC914E175F0745
:101890003CF56B01C20ED31EE6012197D7FD20C097
:1018A0007A01E00EF11ED7011197B7FD19C077FF3D
:1018B00003C0960170E060E057FF03C0870150E06D
:1018C00040E0CA15DB051CF09501261B370BAE174F
:1018D000BF071CF08F01041B150B74010E947009D7
:1018E000DF91CF911F910F91FF90EF90DF90CF90FC
:1018F000BF90AF909F908F900895EF92FF920F93BB
:101900001F93CF93DF93EC0177FD22C088859985E3
:1019100068177907ECF457FD1BC08A859B8548172B
:101920005907B4F47901E881F98102A4F3A5E02D07
:1019300001E010E021E030E0CE010995B701CE01D1
:10194000DF91CF911F910F91FF90EF900C941A08A7
:10195000DF91CF911F910F91FF90EF900895CF935A
:10196000DF93EC010E94FA088FA987FD06C0EB8D7A
:10197000FC8D80819AA989238083DF91CF9108957E
:1019800008950F931F93CF93DF93EC018B010E9477
:10199000FA088FA987FD06C0EB8DFC8D80819AA97E
:1019A00089238083ED8DFE8D80819CA9892380838E
:1019B00066E3CE010E945B08ED8DFE8D80819BA9C0
:1019C000892B80838DA9F801823091F06081CE014E
:1019D0000E945B088FA987FD06C0EB8DFC8D80817E
:1019E00099A9892B8083DF91CF911F910F91089541
:1019F00088A9882359F360817181CE010E941A0859
:101A0000E9CFCF93DF931F92CDB7DEB7FC011982E8
:101A10006370668BDC01AD5BBF4F2C9130E011969B
:101A20008C9190E0623031F06330C9F0613081F028
:101A300040EC498332AF21AF94AF83AFBE016F5FFB
:101A40007F4FCF010E94C10C0F90DF91CF9108957D
:101A500040EA498334AF23AF92AF81AFEFCF40E686
:101A6000F8CF0F931F93CF93DF931F92CDB7DEB7BD
:101A7000FC0119826370668BDC01A85BBF4F2D915E
:101A80003C91119712968D919C916230D1F1633007
:101A900009F440C08F010C5B1F4F6130F9F040EC3E
:101AA0004983AF014D5B5F4FDA014C9150E052AF7B
:101AB00041AFD8014C9150E054AF43AF31872087FC
:101AC00093878287BE016F5F7F4FCF010E94C10C59
:101AD0000F90DF91CF911F910F91089540EA4983B4
:101AE000D8014C9150E052AF41AFDF01AA5BBF4F2C
:101AF0004C9150E054AF43AF338722879187808762
:101B0000E1CFDF01AA5BBF4F4C9150E052AF41AF34
:101B10001196D0CF40E64983DF01A95BBF4F4C91BE
:101B200050E052AF41AF1497E3CFFC0187A987FD86
:101B300006C0A38DB48D9C9181A9892B8C930895A7
:101B40000895FC016370668B8481958126813781BD
:101B5000613039F0633029F091878087338722879D
:101B60000895318720879387828708952F923F9227
:101B70004F925F926F927F928F929F92AF92BF929D
:101B8000CF92DF92EF92FF920F931F93CF93DF9349
:101B9000CDB7DEB76A970FB6F894DEBF0FBECDBFE4
:101BA0009A8F898F7A8369834A01D22E18870F838F
:101BB0003701BC2CDC0159962D913C915A97211587
:101BC000310509F015C118968D919C9119976817E8
:101BD00079070CF0D7C11A968D919C914817590737
:101BE0000CF0D0C14C2C512CB6E0CB9E600D711D79
:101BF00011247C876B87161617060CF0C3C1EA2DDB
:101C0000F0E0FA87E98793E0EE0FFF1F9A95E1F77E
:101C1000F88BEF87CF01840F951F181619060CF06B
:101C2000B1C1A98DBA8D58968C91811104C0BFEABB
:101C3000BD1508F4D394A98DBA8DED91FC9111973F
:101C40000284F385E02DCD010995B5E0DB9EC0014E
:101C50001124E981FA81FC83EB83312C212C9C0136
:101C600020553D4F388F2F8B4A2D50E05E8B4D8B8A
:101C7000EF89F88DE20DF31D44919E828D82D12C67
:101C8000C12C69817A81620D731D7A8B698B842FD7
:101C900090E09C8B8B8BE98DFA8DA081B18140FF08
:101CA00082C0F1E0BF126FC0AF126DC01C96ED9103
:101CB000FC912F813885A4014C0D5D1D69897A89BD
:101CC000898D9A8D0995EB89FC89F595E7954E2FBD
:101CD0005FEFC51AD50A6D817E818D899E89680F57
:101CE000791F7E836D8398E0C916D10481F6AFEF2A
:101CF0002A1A3A0AEB81FC81E40DF51DFC83EB8383
:101D0000F5E02F16310409F0B3CF2F813885261561
:101D10003705B9F0A98DBA8DED91FC91B1E0BB12F8
:101D200057C0AB1255C069817A816B5F7F4F0088C5
:101D3000F189E02D830128E030E0A401898D9A8D9E
:101D40000995A98DBA8DED91FC9111970688F789B7
:101D5000E02DCD016A960FB6F894DEBF0FBECDBF61
:101D6000DF91CF911F910F91FF90EF90DF90CF9077
:101D7000BF90AF909F908F907F906F905F904F90AB
:101D80003F902F9009941E96ED91FC91EF80F8847E
:101D900009851A8592014D815E816B817C81898DD7
:101DA0009A8D099590CF2F8138852615370509F42E
:101DB0008ACF31E0B31207C0A31205C01C96ED9183
:101DC000FC91930178CF1E96ED91FC917301E0CFC9
:101DD0006B857C85641975090684F785E02D730190
:101DE0000F8518899201A401898D9A8D0995A9CF33
:101DF000F90134969491329745915491D91AB7E0EC
:101E0000DB9E400D511D1124F901259134913C8B2D
:101E10002B8BFA0125903490FA013296749031960A
:101E20003491398B329664903196449041E04C1550
:101E300018F04A1508F07FC0662D062C000C770BB1
:101E40007C836B83842D042C000C990B9E838D83E3
:101E5000A98DBA8DED91FC9111970284F385E02D47
:101E6000CD010995512CD12CC12CEA2DF0E0FA8737
:101E7000E9872B2D30E03C872B87A401440D511DB1
:101E800047FC5A95588F4F8B69817A81660D711D79
:101E900067FC7A957E876D877989C71608F051CFE0
:101EA0002C2D30E04D815E81420F531FA985BA85EC
:101EB0004A9FC0014B9F900D5A9F900D1124FC0129
:101EC000E80DF91DF88BEF87852D612C4F89588D12
:101ED000420F531F5E8B4D8B671408F050C0442493
:101EE0004394480E877041F4C1010196EB89FC8947
:101EF000E20DF31DD4901C01D7FE19C0A98DBA8D37
:101F0000ED91FC91662D70E0B1E0BB1219C0AB12EF
:101F100017C02D853E85620F731F0484F585E02D63
:101F20002F8138854D895E89898D9A8D0995DD0CC3
:101F30006394842DD1CF1E821D821C821B8288CF88
:101F40004B815C81640F751FAB85BC856A9FC001A6
:101F50006B9F900D7A9F900D112469817A81680F93
:101F6000791F0684F785E02DEF80F88409851A85AE
:101F70009D014F855889898D9A8D0995D8CF570C29
:101F8000C3948ACF6A960FB6F894DEBF0FBECDBF5A
:101F9000DF91CF911F910F91FF90EF90DF90CF9045
:101FA000BF90AF909F908F907F906F905F904F9079
:101FB0003F902F9008958F929F92AF92CF92EF9281
:101FC000FF920F931F93CF93DF93EC01262F898D00
:101FD0009A8D009709F051C06A30D1F41D861C8695
:101FE0008D8948E0849F900111248E859F85820F02
:101FF000931F9F878E8781E090E0DF91CF911F91A3
:102000000F91FF90EF90CF90AF909F908F90089599
:102010006D3089F3CC88AD888F898823C1F08C8599
:102020009D8536E0C39E800D911D112448855985FC
:102030004817590764F44E855F851D861C8638E075
:10204000A39EC0011124840F951F9F878E87EA8865
:10205000FB88088919894E855F856C857D85CE0151
:102060000E94B60D2C898C859D8546E0249F800DAD
:10207000911D11249D878C87BECF6A3069F41D861F
:102080001C86FC013896E4912D898E859F85E29F00
:10209000800D911D1124ADCF6D3009F4ACCFFC0142
:1020A00034963491631708F4A6CF3296E491E6177C
:1020B00008F4A1CFFC01329685909490462F431BE3
:1020C000342F47E0349F800C911C1124F401329688
:1020D00034913196E4913323A9F1EE2399F1CC8820
:1020E000F4013596E491AD884F89442301F10E2E19
:1020F000000CFF0BE30FF11DCE9EA001CF9E500DF3
:1021000011246C857D85460F571F68857985641776
:1021100075076CF44E855F851D861C86FC0138961C
:10212000E491AE9E400D511D11245F874E87EA88D1
:10213000FB88088919894E855F856C857D85CE0170
:102140000E94B60DF4013496E4912C898C859D850E
:10215000E29F800D911D11248DCF6F927F928F92FF
:102160009F92AF92BF92CF92DF92EF92FF920F9326
:102170001F93CF93DF93EC016B015A0139014801A2
:10218000E881F9810284F385E02D0995E881F981E0
:102190000288F389E02D87019301A501B601CE01E4
:1021A0000995A501480D591D41505109E881F98152
:1021B0000288F389E02D9301B601CE010995E881EB
:1021C000F9810088F189E02D9401A501B601CE01C5
:1021D0000995C60CD71CB60161507109E881F981D7
:1021E0000088F189E02D9401A501CE010995E881CF
:1021F000F9810688F789E02DCE01DF91CF911F91FB
:102200000F91FF90EF90DF90CF90BF90AF909F9095
:102210008F907F906F9009946F927F928F929F9290
:10222000AF92BF92CF92DF92EF92FF920F931F93E4
:10223000CF93DF935C01EB016A014901380187010B
:10224000DC01ED91FC916217730719F564167506B0
:102250002CF0962D872D3A01C92ED82E96012619DD
:1022600037092F5F3F4F048CF58DE02DA301BE0190
:10227000C5010995DF91CF911F910F91FF90EF90CC
:10228000DF90CF90BF90AF909F908F907F906F9096
:1022900008954615570591F42617370724F0892D20
:1022A0004B01C22FD82F9E01281939092F5F3F4FAC
:1022B000068CF78DE02DA601B401DACF0284F385F8
:1022C000E02D0995D501ED91FC910488F589E02D6B
:1022D00083019401A601BE01C5010995D501ED91C7
:1022E000FC910688F789E02DC501DF91CF911F9100
:1022F0000F91FF90EF90DF90CF90BF90AF909F90A5
:102300008F907F906F900994EF92FF920F931F939D
:10231000DC011A960D911C911B9718962D913C91FA
:102320001997ED91FC9100A0F1A1E02D7B0150E007
:1023300040E070E060E009951F910F91FF90EF90F1
:1023400008954F925F926F927F928F929F92AF9279
:10235000BF92CF92DF92EF92FF920F931F93CF9392
:10236000DF936C012B015A0139014801DC01ED9129
:10237000FC910284F385E02D0995E201640C751C43
:10238000D601ED91FC91C615D7055CF40088F18962
:10239000E02D87019401A501BE01C6010995219692
:1023A000EFCF0688F789E02DC601DF91CF911F910D
:1023B0000F91FF90EF90DF90CF90BF90AF909F90E4
:1023C0008F907F906F905F904F9009948F929F9223
:1023D000AF92BF92CF92DF92EF92FF920F931F9333
:1023E000CF93DF93EC015B014A016901E881F98138
:1023F0000284F385E02D099595012C0D3D1D21509A
:102400003109E881F9810488F589E02D780184019A
:10241000A401B501CE010995E881F9810688F78903
:10242000E02DCE01DF91CF911F910F91FF90EF90A2
:10243000DF90CF90BF90AF909F908F9009948F9234
:102440009F92AF92BF92CF92DF92EF92FF920F9343
:102450001F93CF93DF93EC015B014A01690178017F
:10246000E881F9810284F385E02D0995C80CD91C17
:10247000860101501109E881F9810488F589E02D70
:102480009501A401B501CE010995E881F98106887D
:10249000F789E02DCE01DF91CF911F910F91FF9031
:1024A000EF90DF90CF90BF90AF909F908F90099466
:1024B000EF92FF920F931F93DC01ED91FC9100A02E
:1024C000F1A1E02D09951F910F91FF90EF900895D4
:1024D0000F931F93DC01ED91FC91068CF78DE02D9D
:1024E00009951F910F9108950F931F93DC01ED91B2
:1024F000FC91048CF58DE02D09951F910F910895A5
:10250000DC01ED91FC910084F185E02D09942F927E
:102510003F924F925F926F927F928F929F92AF9273
:10252000BF92CF92DF92EF92FF920F931F93CF93C0
:10253000DF9300D000D000D0CDB7DEB73C016A01F8
:102540003E832D83FC82EB825801A41AB50AB7FEA4
:1025500003C0B194A194B1088D809E80861A970A19
:1025600097FE03C09194819491088A149B045CF0B7
:10257000902F812F0D811E819D838E839C2D8D2D0B
:102580006B01692F782F0C151D055CF09D818E81E4
:102590007E836D83692F782F902F812F8601C92E1E
:1025A000D82E1601201A310A2B012D813E81421AA4
:1025B000530A57FE03C0519441945108710137FEEC
:1025C00003C03FEFE31AF30AF594E7948D819E81EF
:1025D000861797075CF5A1E0B0E0BA83A983C0161F
:1025E000D1064CF1D301ED91FC910484F585E02DE9
:1025F0002B813C81A8016D817E818A149B041CF093
:102600004D815E81B801C3010995E418F508F7FE14
:102610000AC02D813E8189819A81280F391F3E830E
:102620002D83E20CF31C0F5F1F4FD9CF2FEF3FEF2D
:102630003A832983D4CF26960FB6F894DEBF0FBE17
:10264000CDBFDF91CF911F910F91FF90EF90DF9061
:10265000CF90BF90AF909F908F907F906F905F9042
:102660004F903F902F900895089590E080E0089556
:10267000CF92DF92EF92FF920F931F93CF93DF934E
:10268000EC01088119816A817B81601B710B072E27
:10269000000C880B990B0E94F9319B01AC0160E0A2
:1026A00070E080EC91E40E944F316B017C01688501
:1026B0007985601B710B072E000C880B990B0E940B
:1026C000F9319B01AC01C701B6010E9406336B01D1
:1026D0007C0120E030E0A9010E94013320E030E0DD
:1026E00040E05FE387FD0BC0C701B6010E94DE300A
:1026F0000E94C13177FF08C0645F7F4FFBCFC701E5
:10270000B6010E94DD30F4CFCB016CE070E00E9496
:10271000FA34FC01EE0FFF1FE158FE4F80819181DA
:102720000197DF91CF911F910F91FF90EF90DF9074
:10273000CF900895CF92DF92EF92FF920F931F9365
:10274000CF93DF936C019A018BE1869FE001879F15
:10275000D00D1124F12CE12C0BE110E0AE01B601FB
:102760008FEA94E00E94A00AEFEAF4E0D586C486DE
:102770002396D787C687DF91CF911F910F91FF9046
:10278000EF90DF90CF90089580912A0190912B01D6
:10279000892B09F054C08091730390917403A09128
:1027A0007503B09176030196A11DB11D809373034B
:1027B00090937403A0937503B093760380910D01F9
:1027C00090910E01409173035091740360917503D1
:1027D00070917603092E000CAA0BBB0B4817590702
:1027E0006A077B0748F081E090E09093DC038093D8
:1027F000DB038093D903089580910D0190910E0120
:102800004091730350917403609175037091760346
:1028100097FD019695958795092E000CAA0BBB0B89
:10282000481759076A077B0750F08091DB039091A6
:10283000DC03892B21F01092DC031092DB03089556
:10284000DC01ED91FD918081ED91FD919081ED9103
:10285000FD916C9163708E2309F064609F2309F0F1
:102860006860EDE3F4E1E60FF11D659565956D9304
:102870006D917D918D919D91099423C01AC012C0D4
:1028800016C010C01EC009C014C013C006C019C0B5
:1028900009C00DC007C00DC014C062507040804018
:1028A00090400BC0615070408040904006C06E5F09
:1028B00001C06F5F7F4F8F4F9F4F9E938E937E938C
:1028C0006E9308958091F4029091F5020C94201477
:1028D0008091F2029091F3020C942014CF93DF9335
:1028E000EC018B85823060F4F894CE010E942014B4
:1028F0006F81788589859A857894DF91CF91089545
:10290000F894F6CF8F929F92AF92BF920F931F933E
:10291000CF93DF93CDB7DEB7A1970FB6F894DEBFA4
:102920000FBECDBF19A2423008F44AE08E010F5D00
:102930001F4F842E912CB12CA12CA50194010E9433
:10294000AC30E62FB901CA01EA3044F5E05DD801A8
:10295000EE938D01232B242B252B79F790E080E03B
:10296000109769F0FD0101900020E9F73197AF0160
:102970004A1B5B0BBD018FEA94E00E945806A196AA
:102980000FB6F894DEBF0FBECDBFDF91CF911F9180
:102990000F91BF90AF909F908F900895E95CD7CF33
:1029A000CF92DF92EF92FF92CF93DF936B017C0186
:1029B0006DE28FEA94E00E94DB0FEC016627772737
:1029C000CB016C197D098E099F094AE00E9482148F
:1029D0008C0F9D1FDF91CF91FF90EF90DF90CF90F4
:1029E0000895009769F0FC0101900020E9F7319704
:1029F000AF01481B590BBC018FEA94E00C945806B8
:102A000090E080E00895AF92BF92CF92DF92EF9274
:102A1000FF920F931F93CF93DF937C018B01EA0109
:102A2000219740EF50E063E070E08AE090E00E9480
:102A30009A13C7010E94F11499E1A92E9CEFB92EB7
:102A40008091F0039091F1030E946E146B01960146
:102A500021703327232B09F596012A193B091216F9
:102A60001306C4F16A157B05C1F08FEF9FEFC80F05
:102A7000D91FD7FF32C0229644E650E063E070E0F1
:102A800080EA90E00E949A13FE01EE0FFF1FE00F14
:102A9000F11F808191810E94F1148091EE03909149
:102AA000EF030E948E06E091EE03F091EF03808524
:102AB00080FD0EC082FF0CC0CE01DF91CF911F912F
:102AC0000F91FF90EF90DF90CF90BF90AF9008955F
:102AD0005601B6CF81E090E0CACFC230D10561F691
:102AE000D0E0C0E0C9CFCF92DF92EF92FF92209169
:102AF000C103211156C041110EC0C090F602D09002
:102B0000F702E090F802F090F902C616D706E80640
:102B1000F90609F446C06B017C01C092F602D0921E
:102B2000F702E092F802F092F9024CE350E064E020
:102B300070E08CE390E00E949A1380912A019091BA
:102B40002B01892B79F081EBC81684E0D806E104CB
:102B5000F10444F08DEF91E0FF90EF90DF90CF9083
:102B60000C94F114F7FE17C0C701B6010E94D014EF
:102B700020E030E040E85FE36091180170911901B6
:102B800080911A0190911B010E944A31882349F0DB
:102B90008FEF91E0E1CF4AE0C701B6010E948214B5
:102BA000E7CFFF90EF90DF90CF900895BC01990F91
:102BB000880B990B97FD0C94D0144AE00C94821466
:102BC000EF92FF920F931F93CF93DF930097A9F09B
:102BD00040912C0150912D0160912E0170912F0197
:102BE0004D3D55406105710544F020910001309143
:102BF00001012F3F3F4F09F450C02091C80430918C
:102C0000C904232B51F42091BD043091BE042A5FE6
:102C10003F4F3093BE042093BD0427EA32E0309347
:102C2000C9042093C8041816190624F5EC018091F4
:102C30002C0190912D01A0912E01B0912F018D3D7D
:102C40009540A105B10584F1E090FA02F090FB02F5
:102C50000FE310E028E330E048E350E066EB70E07B
:102C60008FEA94E00E941B0A8FEF9FEF909301017F
:102C7000809300018091C8049091C904892B49F088
:102C80008091BD049091BE0406979093BE048093FA
:102C9000BD041092C9041092C804DF91CF911F9116
:102CA0000F91FF90EF9008958091000190910101A4
:102CB0008C179D07F9F2E090FF02F09000030FE3FC
:102CC00010E028E330E048E350E066EB70E08FEA84
:102CD00094E00E941B0A8CEB90E09093BC048093DC
:102CE000BB048EE690E09093BE048093BD04CE01B9
:102CF0000E94D615D0930101C0930001BBCFEF9283
:102D0000FF920F931F93CF93DF938C018091250146
:102D1000909126019801281B390B8017910704F523
:102D2000C9011093260100932501EC0121978091A0
:102D3000B903882321F060E083E10E947405F12C3F
:102D4000E12C61E083E1EC16FD066CF40E94740551
:102D500060E083E10E9474053FEFE31AF30AF1CFCC
:102D6000C9010896DECF0E9474050E94F3056093A6
:102D7000B5037093B6038093B7039093B80381E0D3
:102D80008093B903C8010196DF91CF911F910F91F4
:102D9000FF90EF900C94E015CF93DF93EC014CE0A3
:102DA00050E061E070E080EC90E00E949A131C1605
:102DB0001D062CF4CE01DF91CF910C94D615DF9136
:102DC000CF910895CF93DF938091F403C0912101B7
:102DD000D0912201882311F0C6E0D0E08FEF9FEF61
:102DE0009093C2048093C1049093C0048093BF0465
:102DF00082E08093C3048093C40440EA50E061E021
:102E000070E090E080E00E949A13CC0FDD1FC55562
:102E1000DE4F888199810E94F11484EB90E09093B9
:102E2000BC048093BB04CEE1D0E0D093BE04C09339
:102E3000BD0481E092E00E94F1148CEC90E090934C
:102E4000BC048093BB04D093BE04C093BD0483E054
:102E500092E00E94F11480912301909124010E943C
:102E6000CC1690E080E0DF91CF910C94E01580E0EB
:102E700008950F931F93CF93DF93EC01062F142F28
:102E800062E0802F0E94A20562E0812F0E94A205CD
:102E9000802F90E0FC01E75EF74FE491F0E0EE0F49
:102EA000FF1FE352F84FA591B491B983A883FC01A9
:102EB000E550F84F24912C83812F90E0FC01E75ED0
:102EC000F74FE491F0E0EE0FFF1FE352F84F45910A
:102ED00054915B834A83FC01E550F84FE491ED8304
:102EE0001F82188619861A868BE39FE10197F1F7F6
:102EF0008C91282391E009F490E0DA018C91E82389
:102F000009F092609E83BE01802F0E943717082F20
:102F1000BE01812F0E943717800F8B87DF91CF91E1
:102F20001F910F910895809121019091220182308B
:102F3000910511F128F40197A1F090E080E016C00E
:102F400084309105E9F00597C1F70E949C2F892FE5
:102F5000990F990B60912301709124010E94FA341A
:102F600005C08091230190912401019710922901BD
:102F7000109228010C947F1681E080932701DDCF09
:102F80008091310190913201F1CF0E944836CF9269
:102F9000DF92EF92FF920F931F93CF93DF93EC0199
:102FA0006A017B01C114D104E104F10439F4C12C9C
:102FB00048E4D42E48EEE42EFF24F394FE01FF965D
:102FC000C082D182E282F38281E28DAF80E28EAF55
:102FD000369610818FA987FD07C061E00E94A20587
:102FE00061E08FA90E94740561E088AD0E94A2058E
:102FF00061E088AD0E9474058DA9811182C040E016
:1030000052E16AE770E0C416D506E606F70640F41A
:1030100076956795579547958F5F8630A1F787E03E
:10302000212F2C702065982F9695922B99A380952F
:1030300081708AA3812F90E0B0E0A0E08BA39CA3D5
:10304000ADA3BEA31FB7F89480917203811127C06E
:10305000E3E2F8E08491E5E0F8E09491E82FF0E015
:10306000EE0FFF1FED52F84FA591B491EC91E923BB
:1030700021F461E08AE00E94740561E08AE00E9428
:10308000A2058CB580618CBD8CB580648CBD61E07F
:103090008DE00E94A20561E08BE00E94A205809174
:1030A00072038F5F809372031FBF8EA987FD75C067
:1030B00061E00E94A20561E08EA90E94740564E6A9
:1030C00070E080E090E00E94180660E08EA90E9407
:1030D000740564E670E080E090E00E94180661E00C
:1030E0008EA90E94740568EC70E080E090E0DF91AA
:1030F000CF911F910F91FF90EF90DF90CF900C94A4
:10310000180609E118E0F12C8130B9F461E08AA5D4
:103110000E94A20560E08AA50E94740561E08CA56A
:103120000E94A20560E08CA50E9474058BA587FD16
:10313000BCCF60E00E94A205B8CFF8018491E82FCF
:10314000F0E0EE0FFF1FE15FF74F859194912F8D17
:1031500038A12817390741F461E08F2D0E94A2059C
:1031600060E08F2D0E947405F3940F5F1F4FF4E110
:10317000FF12E3CF61E08EA50E94A20561E08EA55B
:103180000E9474058FA587FD90CF61E00E94A20583
:1031900061E08FA50E94740588CFDF91CF911F91C8
:1031A0000F91FF90EF90DF90CF9008951F93CF93F2
:1031B000DF9385ED8093BC0080910403909105031B
:1031C000A0910603B09107030796A11DB11D23E04E
:1031D000B695A795979587952A95D1F72091BC002C
:1031E00024FD03C010924C0352C04091040350913F
:1031F00005036091060370910703452B462B472B6F
:1032000069F30097A105B10541F02AE22A95F1F78B
:1032100000C00197A109B109E1CF80910303C1E08A
:10322000C0930203882399F1D091B8001091BA009D
:103230008091BC008A7B8093BC0060E082E10E94A8
:10324000740560E083E10E94740510924C03C09302
:103250004E0310924D0361E082E10E94740561E02B
:1032600083E10E9474058091B9008E7F8093B9003C
:103270008091B9008D7F8093B90088E48093B80075
:1032800085E48093BC001093BA00D093B800DF911E
:10329000CF911F9108950F931F93CF93DF938C01CC
:1032A000EB010E9450308883C80101960E94503083
:1032B0008983CE01DF91CF911F910F91089590E006
:1032C0000C945030882349F086E00E945F1991E009
:1032D000811101C090E09093FC028091FC022FE1EB
:1032E00030E0882311F020E038EF30930003209382
:1032F000FF0220EE3FEF882311F02FEF3FEF3093D6
:10330000FE022093FD02811107C08AE090E09093B5
:10331000FB028093FA02089580E090EAF8CFFF92D2
:103320000F931F93CF93DF938C01EB01F8800E94E2
:103330005030F81621F06F2DC8010E945830CE0190
:10334000DF91CF911F910F91FF900895FF920F93FE
:103350001F93CF93DF93EC018B01FB01F0800E9460
:103360005030F81621F06F2DCE010E945830F80130
:10337000F1802196CE010E945030F81621F06F2D79
:10338000CE010E945830C801DF91CF911F910F915B
:10339000FF900895CF92DF92EF92FF920F931F93C9
:1033A000CF93DF93CDB7DEB728970FB6F894DEBF83
:1033B0000FBECDBFD82E81E00E9462191092C103CA
:1033C00070E060E08FEA94E00E94841180910C012B
:1033D00061E0811163E08FEA94E00E94310DE0909A
:1033E000FF02F09000030DE110E020EF30E050E02C
:1033F00040E070E060E08FEA94E00E941B0A8FEFEB
:103400009FEF9093C2048093C1049093C004809373
:10341000BF048CE390E09093BC048093BB0485E0F0
:1034200090E09093BE048093BD0482E08093C30437
:103430008093C40485E092E00E94F114DD2009F439
:1034400028C18AE090E09093BC048093BB048EE195
:1034500090E09093BE048093BD0480E192E00E94CE
:10346000F11468EE73E080E090E00E94180684E0BA
:103470000E945F1991E0811101C090E090931C01BE
:103480008AE00E945F1991E0811101C090E0909361
:10349000960380918B0390918C030E948E068091FD
:1034A000EE039091EF030E948E06E091EE03F091FF
:1034B000EF03808580FD64C140EF50E062E070E082
:1034C0008AE090E00E949A1385E192E00E94F11454
:1034D00080918B0390918C03FC01208520FF07C015
:1034E000E091EE03F091EF03208520FD09C00E94DA
:1034F0008E068091EE039091EF030E948E06E8CF36
:1035000080914F0190915001A0915101B0915201D1
:103510008D839E83AF83B88740911C0181E048274B
:1035200050E0BE016B5F7F4F83E292E00E94031583
:1035300021E0892B09F020E020931C016CE171E06F
:1035400084E090E00E948F19809153019091540182
:10355000A0915501B091560189839A83AB83BC83B6
:103560004091FC0250E0BE016F5F7F4F80E392E02C
:103570000E94031521E0019709F020E02093FC024E
:103580006CEF72E086E090E00E948F194091960304
:1035900081E0482750E0BE016B5F7F4F88E392E0F7
:1035A0000E94031521E0892B09F020E02093960367
:1035B00066E973E08AE090E00E948F1980E00E9443
:1035C000CA19BE016B5F7F4F90E080E00E944B19EB
:1035D0008D819E811816190624F49093050180931D
:1035E0000401BE016F5F7F4F82E090E00E944B19A3
:1035F00089819A811816190624F490930301809307
:10360000020187E190E00E942335FC012091020134
:103610003091030140910401509105018FEF9FEF1C
:103620009487838796878587948B838B88E090E047
:10363000968B858B5183408333832283118610863A
:1036400082E090E09583848384E190E09783868391
:10365000F093C703E093C603E0919103F0919203C6
:10366000F89417821086118612867894E091F00300
:10367000F091F103F89417821086118612867894DF
:1036800087E090E0909388038093870380E00E9416
:1036900062191092BC041092BB0404E510E0109370
:1036A000BE040093BD0484E792E00E94F1141092DE
:1036B000BC041092BB048FE690E09093BE0480930C
:1036C000BD0480E892E00E94F1140E94E21680910D
:1036D0002301909124010E94CC1684E890E09093FD
:1036E000BC048093BB041093BE040093BD0488E027
:1036F00090E00E94D6158FEF9FEF90932B0180935F
:103700002A010E94CD1CE090FF02F090000303E428
:1037100010E02CE330E046E350E064EB70E08FEA29
:1037200094E00E941B0AE090FD02F090FE022CE360
:1037300030E046E350E064EB70E08FEA94E00E94F2
:10374000AD10E090FD02F090FE0201E410E02AE3EB
:1037500030E047E350E065EB70E08FEA94E00E94D0
:10376000AD1028960FB6F894DEBF0FBECDBFDF9127
:10377000CF911F910F91FF90EF90DF90CF90089520
:10378000E0918B03F0918C03808580FD1ACF40EF90
:1037900050E061E070E090E080E00E949A1384E4E1
:1037A00092E00E94F11480918B0390918C03FC01B4
:1037B000208520FF07C0E091EE03F091EF03208504
:1037C00020FD09C00E948E068091EE039091EF03C8
:1037D0000E948E06E8CF1092BC041092BB0489E3CD
:1037E000E82EF12CF092BE04E092BD048EE492E04B
:1037F0000E94F11460ED77E080E090E00E941806EE
:1038000084E10E94DE050FEF13E09801281B390BBD
:103810003E832D8398E7C92ED12CD092BC04C09250
:10382000BB04F092BE04E092BD0486E592E00E94E3
:10383000F1148D819E810E94D6158BE592E00E9445
:10384000F11468EE73E080E090E00E941806109298
:10385000BC041092BB0424E5E22EF12CF092BE04CD
:10386000E092BD048DE592E00E94F11460ED77E0F6
:1038700080E090E00E94180684E10E94DE05F801D5
:10388000E81BF90BCF01FA83E983D092BC04C09204
:10389000BB04F092BE04E092BD040E94D6158D8157
:1038A0009E818D599F4F29813A8182179307DCF0C1
:1038B00084E10E94DE059801281B390B3A83298395
:1038C00044E650E063E070E088E790E00E949A13DD
:1038D00089819A810E94D61564E670E080E090E0CC
:1038E0000E941806DCCF88E790E09093BC04809398
:1038F000BB048FE690E09093BE048093BD0485E600
:1039000092E00E94F1141092BC041092BB048AE869
:1039100090E09093BE048093BD048D819E81843895
:103920009340B4F589819A81883E93408CF588E66E
:1039300092E00E94F1148D819E8190930501809305
:10394000040189819A81909303018093020164E0CC
:1039500071E090E080E00E94A61962E071E082E0F0
:1039600090E00E94A61968EB7BE080E090E00E9466
:103970001806F12CE12C07E810E020EF30E04CE1D4
:1039800050E070E060E08FEA94E00E941B0A19CEDC
:103990008DE692E00E94F114E6CFEF92FF920F9332
:1039A0001F9382E10E944B0521E030E0892B11F446
:1039B00030E020E080912A0190912B01821793073B
:1039C00009F477C030932B0120932A0160E081E055
:1039D0000E94740560E083E10E947405F12CE12CE3
:1039E0000BE110E028E730E04CE650E06CE370E0DB
:1039F0008FEA94E00E941B0A88E790E09093BC0451
:103A00008093BB048FE690E09093BE048093BD0446
:103A100080912A0190912B01009741F1019709F4BF
:103A200043C01092D7031092D60310921D0110923A
:103A30001E0110921F011092200180911C01882309
:103A4000C1F10E944B066093C2037093C30380933D
:103A5000C4039093C5038091C103882351F180E092
:103A60001F910F91FF90EF900C94CA1986E992E094
:103A70000E94F11460912C0170912D0180912E0112
:103A800090912F010E94F931209118013091190174
:103A900040911A0150911B010E944F310E94C13187
:103AA00041E00E947315BDCF8BE992E00E94F114B2
:103AB000B8CF1F910F91FF90EF90089580912A0148
:103AC00090912B010197F1F582E00E944B0521E0D6
:103AD00030E0892B11F030E020E03093DC032093BC
:103AE000DB0382E00E944B05019761F182E00E94B6
:103AF0004B0521E0892B09F020E0822F90E0909384
:103B0000DC038093DB032093D8038091F4038111BD
:103B100004C08091D8038823A9F080911C018823D8
:103B200089F00E944B066093C2037093C303809395
:103B3000C4039093C5038091C103882319F080E0EA
:103B40000C94CA1908950E944B066093BD037093AC
:103B5000BE038093BF039093C0038091A303909111
:103B6000A40363E070E00E94FA34892B01F564EF4E
:103B700071E080E090E00E94180670E060E08FEA5B
:103B800094E00E94841164EF71E080E090E00E9474
:103B900018060E94F82F23E030E040E050E00E9439
:103BA0007A306E5F7F4F70931101609310010E9415
:103BB000F82F23E030E040E050E00E947A3070932C
:103BC000B4036093B3030E94F82F22E330E040E097
:103BD00050E00E947A30FB014091A5035091A6036A
:103BE0004115510509F47CC04330510509F478C0F2
:103BF0002091B7043091B804261B370B3093A803EB
:103C00002093A7034230510534F0E091B904F091BC
:103C1000BA04E61BF70BF093AA03E093A9032091E3
:103C2000B7043091B8044230510514F430E020E07C
:103C30003093B2032093B1034115510529F030E0D0
:103C400020E04330510521F42091B9043091BA04A9
:103C50003093AE032093AD032091B7043091B804A4
:103C60004230510514F030E020E03093B00320934F
:103C7000AF034115510539F04330510599F1409199
:103C8000B9045091BA045093AC034093AB030E9423
:103C9000F82F2DE730E040E050E00E947A30675E78
:103CA0007F4F8F4F9F4F0E94F93120E030E048E472
:103CB00052E40E944F316093140170931501809378
:103CC0001601909317010E94F82F2FEF3FEF40E06D
:103CD00050E00E947A3070931301609312010895AE
:103CE0009B018CCF50E040E0CECF1F920F920FB6D9
:103CF0000F9211242F933F938F939F93AF93BF9372
:103D00008091E6039091E703A091E803B091E90365
:103D10003091E50323E0230F2D3758F50196A11DBF
:103D2000B11D2093E5038093E6039093E703A093EE
:103D3000E803B093E9038091EA039091EB03A0912B
:103D4000EC03B091ED030196A11DB11D8093EA0330
:103D50009093EB03A093EC03B093ED03BF91AF916D
:103D60009F918F913F912F910F900FBE0F901F90B9
:103D7000189526E8230F0296A11DB11DD2CF1F92E0
:103D80000F920FB60F9211242F933F934F935F938F
:103D90006F937F938F939F93AF93BF93EF93FF9313
:103DA000E0910801F09109010995FF91EF91BF9110
:103DB000AF919F918F917F916F915F914F913F91C3
:103DC0002F910F900FBE0F901F9018951F920F927A
:103DD0000FB60F9211242F933F934F935F936F93DE
:103DE0007F938F939F93AF93BF93EF93FF93E09154
:103DF0000601F09107010995FF91EF91BF91AF91F5
:103E00009F918F917F916F915F914F913F912F91F2
:103E10000F900FBE0F901F9018951F920F920FB624
:103E20000F9211242F933F934F935F936F937F9340
:103E30008F939F93AF93BF93EF93FF9385EF93E09F
:103E40000E947F04FF91EF91BF91AF919F918F915D
:103E50007F916F915F914F913F912F910F900FBE86
:103E60000F901F9018951F920F920FB60F9211246A
:103E70002F938F939F93EF93FF93E0910504F0911D
:103E800006048081E0910B04F0910C0482FD1BC0BC
:103E9000908180910E048F5F8F7320910F048217A1
:103EA00041F0E0910E04F0E0EB50FC4F958F8093D1
:103EB0000E04FF91EF919F918F912F910F900FBE64
:103EC0000F901F9018958081F4CF1F920F920FB61C
:103ED0000F9211242F933F934F935F936F937F9390
:103EE0008F939F93AF93BF93EF93FF93E0910A015A
:103EF000F0910B010995FF91EF91BF91AF919F91C7
:103F00008F917F916F915F914F913F912F910F9082
:103F10000FBE0F901F9018951F920F920FB60F9221
:103F200011242F933F934F935F936F937F938F93BE
:103F30009F93AF93BF93EF93FF938091B900887FD6
:103F4000803609F44AC0F0F5883209F4A5C018F5A6
:103F5000803109F499C0B8F4882309F4F5C0883099
:103F600009F492C0FF91EF91BF91AF919F918F9112
:103F70007F916F915F914F913F912F910F900FBE65
:103F80000F901F901895883109F486C0803251F740
:103F900080934B0314C0803409F49BC040F48033F9
:103FA000B9F38833F9F680934B0385ECAEC08035C6
:103FB00009F483C0883509F494C0883499F60E94C6
:103FC000D618D0CF883909F48AC038F5883729F057
:103FD00050F4883611F0803729F683E080934C0343
:103FE00010924A0355C0883809F479C0803919F015
:103FF000803809F0B7CF80914A03803208F06FC053
:10400000E0914A0381E08E0F80934A038091BB00C8
:10401000F0E0E65DFC4F80833BC0803B39F0D0F49C
:10402000803A09F477C0883A09F09CCF84E0809305
:104030004C031092290310922803F0E0E0E0099568
:104040008091280381110FC081E080932803109292
:10405000080309C0803C09F4A8CF883C09F4A5CF27
:10406000883B09F07FCFE091290381E08E0F809398
:104070002903F0E0E85FFC4F80818093BB009091C2
:1040800029038091280329C0809171038093BB008C
:1040900085EC8093BC0066CF9091700380916F0394
:1040A000981758F5E091700381E08E0F80937003AC
:1040B000F0E0E15BFC4F8081E9CFE091700381E0AB
:1040C0008E0F809370038091BB00F0E0E15BFC4FAA
:1040D00080839091700380916F039817C8F285E8F0
:1040E000D8CFE091700381E08E0F809370038091B0
:1040F000BB00F0E0E15BFC4F808380914E038111B7
:104100005ECF81E080934D0384EA8093BC001092DF
:104110004C0328CF85EC8093BC0010924C03809117
:104120004A03803230F4E0914A03F0E0E65DFC4F50
:10413000108260914A0370E08AE293E0F0E0E0E0F0
:10414000099510924A030ECF10924B0338CFE5EF3A
:10415000F3E01382128288EE93E0A0E0B0E0848363
:104160009583A683B7838FEB91E09183808385EC61
:1041700090E09587848784EC90E09787868780EC31
:1041800090E0918B808B81EC90E0938B828B82EC22
:1041900090E0958B848B86EC90E0978B868B118ECC
:1041A000128E138E148EAFEAB4E013961C921E92F8
:1041B000129720EF30E015963C932E93149780E4ED
:1041C00091E017969C938E93169719963C932E9395
:1041D00018971B969C938E931A9756961C925697F7
:1041E0001D961C921E921C971F961C921E921E9743
:1041F00081E055968C93559754968C9354972FEF56
:104200003FEF53963C932E93529751963C932E93A7
:10421000509757968C93579758961C9258975A9642
:104220001C921E925997D5961C92D59789E0D696E6
:104230008C93D6978AE0D7968C93D79788E0D896B8
:104240008C93D897DA961C921E92D997DC961C9282
:104250001E92DB97DD961C92DD97DE961C92DE9710
:104260001092EE041092EF041092F0041092F104F8
:1042700082E994E090969C938E935F97E1E2F8E058
:10428000E491F0E0EE0FFF1FE15FF74F859194910D
:104290005E969C938E935D97E3E0F8E08491D396CD
:1042A0008C93D397E3E2F8E0E491F0E0EE0FFF1F88
:1042B000E15FF74F259134915C963C932E935B9789
:1042C000E5E0F8E0E491D196EC93D197E095D296B1
:1042D000EC93D297E82FE095D496EC93D497109274
:1042E000F2041092F3041092F40481ED91E08D93A6
:1042F0009C931092F5041092F6040E944B06609372
:10430000AB047093AC048093AD049093AE040E9410
:104310004B06EFE9F4E08DEC9CECACE4BDE380836C
:104320009183A283B38380E090E0A0E0B4E484832F
:104330009583A683B783E3E9F4E08AE999E9A9E9DB
:10434000BEE380839183A283B38380E090E0A0EFFB
:10435000B2E484839583A683B7830895CF93DF93D4
:10436000CDB7DEB7E8970FB6F894DEBF0FBECDBF6E
:10437000789484B5826084BD84B5816084BD85B540
:10438000826085BD85B5816085BD80916E0081604C
:1043900080936E00109281008091810082608093F2
:1043A00081008091810081608093810080918000F4
:1043B0008160809380008091B10084608093B1001F
:1043C0008091B00081608093B00080917A00846019
:1043D00080937A0080917A00826080937A00809145
:1043E0007A00816080937A0080917A00806880935F
:1043F0007A001092C1001092F40440E050E0BA013B
:104400008FEA94E00E94C71788E28093F6048093B5
:10441000F30485E38093F20484E38093F50487E852
:1044200090E09093F8048093F70480EF90E09093ED
:10443000FA048093F904E0EBF7E09490E1EBF7E005
:104440009A9488248A94981409F47AC014915F018C
:1044500002E0A00EB11C31968490082D0F778FEAF0
:1044600094E00E94FA088091E60487FD09C0E0917B
:10447000CA04F091CB0480819091E1048923808368
:10448000E091CC04F091CD0480819091E3048923E4
:104490008083612F8FEA94E00E945B08E091CC0456
:1044A000F091CD0480819091E204892B8083F50105
:1044B000D12CC12C10E0C016D106FCF48091E4048C
:1044C0007F01823089F48091DF04882369F0DF0165
:1044D0006D917D917D018FEA94E00E941A08EFEFC3
:1044E000CE1ADE0AF701E7CFBFEFEB1AFB0A6491A1
:1044F0008FEA94E00E945B08F2CF8091E60487FD8A
:1045000009C0E091CA04F091CB0480819091E0044D
:10451000892B8083F501E00FF11F87FE91CF7F018A
:104520000FEFE01AF00A649170E06F3F710511F42B
:1045300064EF71E090E080E00E941806F70180CF00
:1045400060E08FEA94E00E94310D70E060E08FEA55
:1045500094E00E94841182E08093C3048093C40499
:104560008CE00E945F1991E0811101C090E090936E
:104570000C0163E0811101C061E08FEA94E00E94C8
:10458000310D81E00E94621962E082E10E94A20581
:1045900062E084E00E94A20562E085E00E94A2053C
:1045A0008CE090E00E9423358C0145E064E00E949D
:1045B0003917109392030093910362E086E00E9402
:1045C000A20582E190E00E942335FC011282138251
:1045D000148215823AE0C32ED12CD782C68210866F
:1045E0004BE9E42E41E0F42EF182E08290938C03BB
:1045F00080938B0386E0818BCF010E94F706E091C8
:104600008B03F0918C0302E310E01783068362E0D2
:1046100087E00E94A20562E08CE00E94A2058CE087
:1046200090E00E9423355C014CE067E00E9439175E
:10463000B092F103A092F00362E08EE00E94A20526
:1046400082E190E00E942335FC01128213821482E1
:104650001582D782C6821086F182E0829093EF03A2
:104660008093EE038EE0818BCF010E94F706E091EC
:10467000EE03F091EF031783068361E080E10E946F
:10468000A20561E081E10E94A20562E08FE00E9444
:10469000A20561E081E00E94A20582E190E00E9413
:1046A0002335FC011282138214821582D782C682BE
:1046B0001086F182E08290937D0380937C038FE0EB
:1046C000818BCF010E94F706E0917C03F0917D037E
:1046D000178306836091300181E10E94740560E0D8
:1046E00081E00E94740560E080E10E94740561E051
:1046F00083E10E94A20560E083E10E94740562E00C
:1047000082E00E94A2058EE59DE1909307018093CF
:104710000601809169008C7F816080936900E89A2E
:1047200062E083E00E94A20580E180938100109204
:10473000800082E19AE7909387008093860024E1CD
:104740002093810024EC33E130930B0120930A0184
:1047500021E020936F0023E020939503909394032E
:1047600080939303909387008093860083E18093E6
:1047700081000E944B066093C2037093C303809331
:10478000C4039093C503611571058105910511F06E
:104790000E94473080911C0181110E94A31D81E07D
:1047A0000E94CA190E944B066B017C01C092AB04A7
:1047B000D092AC04E092AD04F092AE040091DB0321
:1047C0001091DC038091DD0381110AC081E00115A5
:1047D000110509F080E08093DA0381E08093DD0326
:1047E0008091DA038017110651F0602F81E00E945A
:1047F000740581E0012B09F480E08093DA03809155
:10480000D903882309F445C01092D90380912A0165
:1048100090912B01892B41F520910D0130910E01D2
:104820006091730370917403809175039091760386
:10483000032E000C440B550B0E94AC3060937303A5
:1048400070937403809375039093760388E190E0EE
:1048500090930E0180930D018091BA03882389F013
:104860001092BA030E94931780E090E0892B09F41C
:1048700099CF0E940E05882309F494CF0E9400006E
:1048800091CF80913001882379F381E08093BB033D
:10489000EBCF8091D803882309F46AC080912A0164
:1048A00090912B01019779F48091D803882359F0D6
:1048B0008091BA03882309F452C01092BA030E946F
:1048C00093171092BB031092D803C0901D01D09093
:1048D0001E01E0901F01F090200120E030E0A901CE
:1048E000C701B6010E94013320E030E040E05FE301
:1048F00087FD39C0C701B6010E94DE300E94C13178
:104900006B017C011C141D041E041F040CF0ACCFB1
:104910008091D6039091D7038C339105B4F0092E82
:10492000000CAA0BBB0B8C199D09AE09BF09B7FF80
:1049300007C0B095A095909581959F4FAF4FBF4F01
:104940000397A105B1050CF48FCF40E0C701B60174
:104950000E947315D092D703C092D60385CF81E011
:104960008093BB03B0CFC701B6010E94DD30C6CF34
:104970008091CE0381110DC00E944B066093CA0343
:104980007093CB038093CC039093CD0381E080930D
:10499000CE038091CA039091CB03A091CC03B09138
:1049A000CD030097A105B105A9F0C81AD90AEA0AF2
:1049B000FB0A11EDC11617E0D106E104F10450F035
:1049C0000E94E2161092CA031092CB031092CC03FD
:1049D0001092CD0300917C0310917D03D8011896AD
:1049E0008C9180FD13C00E944B06F801C184D284D3
:1049F000E384F4846C197D098E099F096093780320
:104A00007093790380937A0390937B03C09078032B
:104A1000D0907903E0907A03F0907B03C8010E9464
:104A20008E0680917703811114C180917C0390914F
:104A30007D030E948606811107C0F8ECCF16D104D1
:104A4000E104F1040CF405C180911C01882309F4F0
:104A5000F0C00E944B066093C2037093C30380931F
:104A6000C4039093C5038091C103882309F4E1C076
:104A700080E00E94CA198091C8039091C9030196F1
:104A80009093C9038093C8036BE070E00E94FA34EE
:104A9000892BC9F483E00E944B059C0191E021150C
:104AA000310509F090E080910F01981761F0909323
:104AB0000F01232B41F480913001882309F41CC19C
:104AC00081E08093BA038091C8039091C90367E0A5
:104AD00070E00E94FA34892B61F5809191039091E6
:104AE00092030E946E146B0100918F03109190034A
:104AF0000617170709F44BC1CB0181709927892B41
:104B000009F045C180911C01882309F4F8C00E9476
:104B10004B066093C2037093C3038093C4039093C6
:104B2000C5038091C103882309F4E9C080E00E9495
:104B3000CA1980912A0190912B01892B09F03AC45E
:104B40008091C8039091C9036DE070E00E94FA342F
:104B50008C01892B09F02EC480919B03811105C023
:104B60000E944B0681E080939B0385E10E94DE0555
:104B70001C01A6E02A1A310860E074E0681B790B7A
:104B8000072E000C880B990BB6EF2B16B3E03B06F3
:104B900008F49EC30E94F9316B017C01C092A3040A
:104BA000D092A404E092A504F092A604C0929703C8
:104BB000D0929803E0929903F0929A038091960321
:104BC000882309F4B4C684E1E7E5F1E0DE015596F7
:104BD00001900D928A95E1F784E1EBE6F1E0DE01C8
:104BE000119601900D928A95E1F720E030E040EABD
:104BF00050E4C701B6010E944A3187FDE2C620E0B9
:104C000030E44EE754E4C701B6010E9401334E017F
:104C100039E1830E911C18160CF03DC558E8852E1D
:104C200053E1952EA12CB12C89A69AA6ABA6BCA6C1
:104C3000C3C581E08093770300913001002301F127
:104C400018ECC116D104E104F104D4F481E080939E
:104C5000BA0380917703882309F40DCFE0917C0398
:104C6000F0917D03808580FF06CF1092770310922C
:104C700078031092790310927A0310927B03FBCE93
:104C800011E010271093300188E190E090930E011D
:104C900080930D01612F81E10E947405602F80E1F6
:104CA0000E9474051123E9F01092DC031092DB03DB
:104CB00060E081E00E94740580912A0190912B01AF
:104CC000892B21F680E1809381001092810010925F
:104CD000850010928400809195038061809381000B
:104CE000B5CF20912A0130912B0181E0213031058F
:104CF00009F4ADCF80E0ABCF0E949317E4CEC6019C
:104D0000801B910B1816190664F481E090E0209145
:104D10008D0330918E03820F931F97FF05C0089675
:104D2000FCCF8FEF9FEFF3CF8770992790938E037F
:104D300080938D0340EA50E062E070E090E080E014
:104D40000E949A130E944B0680918D0390918E03CE
:104D500090937F0380937E03863091055CF480EA14
:104D600092E00E94F11480917E0390917F0386303F
:104D7000910548F4880F991FFC01E555FE4F80818D
:104D800091810E94F114D0929003C0928F03809180
:104D90008B0390918C030E948E068091EE0390917C
:104DA000EF030E948E0680918B0390918C030E94EA
:104DB0008606182F8091EE039091EF030E948606DD
:104DC000B82E112389F180911C01882371F00E9473
:104DD0004B066093C2037093C3038093C403909304
:104DE000C5038091C1038111A1CE80918A038111F5
:104DF00010928A031092890380918D0390918E0303
:104E00008730910509F04AC040EA50E061E070E067
:104E100090E080E00E949A1385EA92E00E94F114EB
:104E200010922601109225018091F0039091F103D8
:104E30000E946E146B01009187031091880306177E
:104E4000170709F4A9C0CB0181709927892B09F0B4
:104E5000A3C080911C01882371F00E944B066093CF
:104E6000C2037093C3038093C4039093C5038091DE
:104E7000C10381115BCEC601801B910B1816190668
:104E80000CF064C081E090E02091F2033091F303D4
:104E9000820F931F97FF5DC00896FCCF1092F4031A
:104EA000863091050CF04BC080917E0390917F037A
:104EB00090932201809321018230910599F481E041
:104EC000809327010E94E2168091F403882309F45D
:104ED000ABCF40EA50E062E070E090E080E00E94FA
:104EE0009A13A2CF049771F791E2E92E91E0F92E7F
:104EF00008E010E00E949C2FB8010E94FA34D7010C
:104F00005E962D913C915F97FC01EE0FFF1FEF5CC9
:104F1000FE4F808191815F969C938E935E9733279D
:104F20003183208301501109B2E0EB1AF108011519
:104F3000110501F71092290110922801C3CF21E039
:104F4000069709F020E02093F403BCCF8FEF9FEF8A
:104F50009BCF877099279093F3038093F20349E1E5
:104F600050E063E070E084E890E00E949A13809142
:104F7000F2039091F30301960E94D6158FEF9FEFF5
:104F80009093C2048093C1049093C0048093BF04A3
:104F9000D0928803C092870380912A0190912B01BF
:104FA000019709F4FFC0809186038111FBC0009135
:104FB000EE031091EF03F801808580FDF3C00E949D
:104FC0004B06D80119960D911D912D913C911C977E
:104FD000601B710B820B930B653F7140810591053E
:104FE00008F4E0C081E0809386038091840390916F
:104FF00085030196833091050CF0F1C090938503F1
:1050000080938403E0918403F0918503EE0FFF1FEA
:10501000EE0FFF1FE156FE4F608171818281938107
:105020000E94C131643071050CF0DEC06F5F7F4FAC
:10503000072E000C880B990B0E94F9319B01AC01E3
:1050400060E070E080E89FE30E944F31609380034E
:10505000709381038093820390938303409018019F
:105060005090190160901A0170901B01C09080034C
:10507000D0908103E0908203F090830311E0A701B8
:105080009601C301B2010E944A31811101C010E0B2
:1050900010938903A7019601C301B2010E944A310E
:1050A000882309F47FC0C0921801D0921901E092C0
:1050B0001A01F0921B0160912C0170912D018091D9
:1050C0002E0190912F010E94F9319B01AC0160ECFF
:1050D00071EE84E69CE40E944F31A70196010E9484
:1050E000063320E030E040EC51E40E944F316B0188
:1050F0007C0120E030E0A9010E94013320E030E093
:1051000040E05FE387FD79C0C701B6010E94DE3051
:105110000E94C131A0EAB0E09B01AC010E9499302D
:105120006B017C0124E130E040E050E00E94AC30B3
:1051300021153105E1E04E07510508F063C081E01B
:10514000809395033093940320939303809193036A
:1051500090919403909387008093860080919503AB
:1051600080618093810080912A0190912B01892B8D
:10517000C9F460912C0170912D0180912E019091C4
:105180002F010E94F93120911801309119014091AD
:105190001A0150911B010E944F310E94C13140E021
:1051A0000E947315BB2009F4C4CC80911C01882394
:1051B00071F00E944B066093C2037093C303809307
:1051C000C4039093C5038091C1038111AFCC80913A
:1051D0008603882309F45EC010928603AACC10923D
:1051E0008503109284030ECF63507109072E000CC3
:1051F000880B990B0E94F93129CFC701B6010E9493
:10520000DD3086CF21153105F8E04F07510560F4F8
:1052100082E080939503C701B60120EA30E040E0C8
:1052200050E00E94AC308ECF2115310500E44007DC
:10523000510550F483E080939503C701B60120E047
:1052400035E040E050E0EDCF21153105410511E09A
:10525000510750F484E080939503C701B60120E024
:1052600034E140E050E0DDCF85E0809395032115E7
:1052700031054105544038F4C701B60120E030E55E
:1052800040E050E0CECF8FEF9FEF90939403809358
:1052900093035CCF8091F2039091F30388309105E2
:1052A000A4F497FF02C090E080E0019620912301D2
:1052B000309124012817390709F43BCC909324013D
:1052C000809323010E94CC1634CC88E090E0EECF8E
:1052D0000E94F9314B015C014090A7045090A80452
:1052E0006090A9047090AA042091A3043091A404B2
:1052F0004091A5045091A6042DA73EA74FA758ABF7
:1053000020E030E0A901C301B2010E944A318823A4
:1053100009F48FC12DA53EA54FA558A9C501B4011B
:105320000E94DD306B017C0120E030E0A9010E9489
:105330000133181624F0F7FAF094F7F8F094A70167
:105340009601C301B2010E944A3187FF72C1809267
:10535000A3049092A404A092A504B092A604C090C5
:10536000A304D090A404E090A504F090A60420919A
:105370009703309198034091990350919A03C70184
:10538000B6010E94DD304B015C0120E030E0A90154
:105390000E940133181624F0B7FAB094B7F8B0940D
:1053A00020E030E040E450E4C501B4010E944A31FD
:1053B00087FFFCCB8091C8039091C9036BEB70E031
:1053C0000E94FA34892B11F40E94CD1C8091F403C1
:1053D0008111C5C3312C8091C8039091C90360E14C
:1053E00077E20E94FA34892BA9F480913001882356
:1053F00009F432C48091AB049091AC04A091AD0447
:10540000B091AE048093C2039093C303A093C403EE
:10541000B093C5038091C103882309F4E3C0809150
:10542000BD039091BE03A091BF03B091C003409112
:10543000AB045091AC046091AD047091AE04481B74
:10544000590B6A0B7B0B4F3151056105710508F44F
:10545000C9C04E96A11DB11D8093BD039093BE039C
:10546000A093BF03B093C00380911C01882309F46B
:10547000B9C06091B3037091B403072E000C880B80
:10548000990B0E94F9316B017C016091B904709114
:10549000BA04072E000C880B990B0E94F9319B016E
:1054A000AC01C701B6010E944F312B013C01209194
:1054B00014013091150140911601509117010E947D
:1054C00073334B015C010091B1031091B203C090A2
:1054D000AD03D090AE03E0901201F0901301609103
:1054E000AB037091AC036C197D09072E000C880B7F
:1054F000990B0E94F931A30192010E9406332B01FE
:105500003C01B601DD0C880B990B0E94F9319B011F
:10551000AC01C301B2010E94DE300E94C1312B01F7
:105520006091AF037091B003601B710B072E000CEC
:10553000880B990B0E94F931A50194010E94063352
:105540004B015C01B801110F880B990B0E94F931D6
:105550009B01AC01C501B4010E94DE300E94C13143
:105560004091A9035091AA03E091A703F091A803E9
:1055700082019B01BF018FEA94E00E940C1180918F
:105580001001909111012091B3033091B403280FC1
:10559000391F3093B4032093B3034091B904509161
:1055A000BA04840F951F82179307E4F48091A50332
:1055B0009091A60301962091A3033091A4032F5F3D
:1055C0003F4F3093A4032093A30364E070E00E9454
:1055D000FA349093A6038093A50380911C01811156
:1055E0000E94A31D8091F403882309F46CC30091E9
:1055F000C6031091C703D8011A966C9181E00E94EE
:105600007405F8018285882311F031104CC390E0B5
:1056100080E00E94CC168091BC03811104C090E010
:1056200080E00E94E01581E08093BC038FEF9FEF44
:1056300042C3C0909F04D090A004E090A104F090D9
:10564000A204A701960160E070E080E89FE30E9459
:10565000DD302DA53EA54FA558A90E9406332B018C
:105660003C01A7019601C501B4010E9406339B01CC
:10567000AC01C301B2010E94DE306093A3047093B9
:10568000A4048093A5049093A60469CE85010430F8
:10569000110509F491C058014FEFA41AB40AF4019E
:1056A00081919191A191B1914F018DA79EA7AFA733
:1056B000B8ABBC01CD010E94F9319B01AC01C7011F
:1056C000B6010E944A3187FFE1CFAA0CBB1CAA0C8D
:1056D000BB1CE1E0F0E0EC0FFD1FEA0DFB1D40807C
:1056E0005180628073805801AA0CBB1CAA0CBB1CA1
:1056F00088248394912C8C0E9D1EA80CB91CD50176
:105700006D917D918D919C910E94F9310E94C131E2
:1057100069A77AA78BA79CA7D50154960D911D91D7
:105720002D913C9157970DAB1EAB2FAB38AFC301FA
:10573000B2010E94F9310E94C1314B015C0109A5FF
:105740001AA52BA53CA5801A910AA20AB30A89AA18
:105750009AAAABAABCAAC701B6010E94C1318DA802
:105760009EA8AFA8B8AC681979098A099B0929A92C
:105770003AA94BA95CA90E94EA342DA53EA54FA5E4
:1057800058A9281939094A095B090E947A3089A465
:105790009AA4ABA4BCA4820E931EA41EB51E89A617
:1057A0009AA6ABA6BCA6481459046A047B0424F448
:1057B00049A65AA66BA67CA669A57AA58BA59CA529
:1057C0000E94F9316B017C0106EF201603E03006E0
:1057D00008F400C1C0929704D0929804E092990412
:1057E000F0929A040E94C13100912C0110912D0178
:1057F00020912E0130912F0106171707280739072E
:1058000009F47DC060932C0170932D0180932E01CB
:1058100090932F010E94F9319B01AC0160EC71EE75
:1058200084E69CE40E944F312091180130911901C7
:1058300040911A0150911B010E94063320E030E094
:1058400040EC51E40E944F316B017C0120E030E0DC
:10585000A9010E94013320E030E040E05FE387FDD2
:1058600031C1C701B6010E94DE300E94C131A0EAF9
:10587000B0E09B01AC010E9499306B017C0124E1F6
:1058800030E040E050E00E94AC302115310501E0ED
:105890004007510508F01BC181E0809395033093C8
:1058A0009403209393038091930390919403909396
:1058B00087008093860080919503806180938100AA
:1058C00080912A0190912B01892BC9F460912C01C0
:1058D00070912D0180912E0190912F010E94F9313C
:1058E000209118013091190140911A0150911B012A
:1058F0000E944F310E94C13140E00E947315809197
:105900001C01882309F456CD0E944B066093C20304
:105910007093C3038093C4039093C5038091C10324
:10592000882309F447CD80E00E94CA1943CDC701FE
:10593000B6010E94C1319B01AC01255031094109DA
:105940005109A4E5B1E00E94993027EF33E040E02F
:1059500050E00E947A3069017A01CA01B901675E9C
:105960007F4F8F4F9F4F0E94F93120E030E040E0A1
:105970005FE307EEC0160FEFD006E006F0063CF13D
:105980000E94DE300E94C13148E6842E992493940F
:10599000A12CB12C89A69AA6ABA6BCA66815790540
:1059A0008A059B0524F469A77AA78BA79CA709A55C
:1059B0001AA52BA53CA50E311105210531050CF0CA
:1059C000FBCE3EE1832E912CA12CB12C2DC90E943F
:1059D000DD30D8CF40909B0450909C0460909D0493
:1059E00070909E048090970490909804A0909904E1
:1059F000B0909A048DA69EA6AFA6B8AA20E030E08B
:105A0000A901C301B2010E944A31882371F1A501A5
:105A10009401C701B6010E94DD304B015C0120E01A
:105A200030E0A9010E940133181624F0B7FAB094AF
:105A3000B7F8B094A5019401C301B2010E944A31A4
:105A400087FF13C0C0929704D0929804E092990403
:105A5000F0929A046091970470919804809199044F
:105A600090919A040E943432BDCE8090930490901D
:105A70009404A0909504B0909604A501940160E070
:105A800070E080E89FE30E94DD302DA53EA54FA584
:105A900058A90E9406332B013C01A5019401C701BE
:105AA000B6010E9406339B01AC01C301B2010E9402
:105AB000DE306093970470939804809399049093D8
:105AC0009A04C8CFC701B6010E94DD30CECE2115A1
:105AD000310518E04107510560F482E08093950399
:105AE000C701B60120EA30E040E050E00E94AC304F
:105AF000D6CE2115310580E44807510550F483E0E6
:105B000080939503C701B60120E035E040E050E006
:105B1000EDCF21153105410591E0590750F484E09E
:105B200080939503C701B60120E034E140E050E0E6
:105B3000DDCF85E080939503211531054105544063
:105B400038F4C701B60120E030E540E050E0CECFA8
:105B50008FEF9FEF9093940380939303A4CE0091D3
:105B6000C6031091C7030E944B062B013C01F801AC
:105B700084810E944B0521E0019709F420E0D801BF
:105B80001A962C931A9716968C910E94DE052FEF89
:105B900033E0281B390BF80131872087328431101C
:105BA0000DC01786108A118A128A8FEF9FEF948B8F
:105BB000838B96878587118610860DCC8785908983
:105BC000A189B289892B8A2B8B2B21F44786508A95
:105BD000618A728AF801E384F484F686E586C80156
:105BE0000E943813D8011C969C938E931B971F9686
:105BF0004D915D916D917C915297411551056105D3
:105C0000710509F4E7CB441A550A660A770A5596D6
:105C10002D913C915697032E000C440B550B2415E7
:105C200035054605570508F0D5CB53962D913C9187
:105C30008217930709F4CECBE816F90609F0CACB10
:105C4000F8011786108A118A128AF48AE38A8FEF84
:105C50009FEF96878587BFCB80911C01882309F42D
:105C6000D9CB8091C1038111DACB0E944B06009100
:105C7000C2031091C3032091C4033091C503601B7C
:105C8000710B820B930B613E73498440910508F4BC
:105C9000A9CC81E08093C10370E060E08FEA94E0DA
:105CA0000E948411B7CBC8010E94381321E02093D1
:105CB000BB031092BC032091BA03222339F0109247
:105CC000BB030C94342490E080E0F5CF2091D803FE
:105CD00021110C94342420913001211106C020910F
:105CE000F403222311F40C9434242091BB032223C7
:105CF00061F01092BB0321E02093B9032091F403DB
:105D0000222309F453C00E947F1660912C017091E8
:105D10002D0180912E0190912F0122E030E040E092
:105D200050E00E947A30CA01B9010E94F9312091F5
:105D300018013091190140911A0150911B010E94E4
:105D40004F3120E030E44CE955E40E94013308EC87
:105D500010E087FF02C008E512E08091B9038823B4
:105D600011F40C9434240E94F305AB01BC01C8016A
:105D7000110FAA0BBB0B0091B5031091B603209134
:105D8000B7033091B803800F911FA21FB31F4817AC
:105D900059076A077B0710F40C9434241092B90356
:105DA00060E083E10E9474050C9434240091230187
:105DB00010912401209121013091220123303105DD
:105DC00009F447C0B0F4809125019091260121305B
:105DD0003105F9F02230310531F1809125019091A2
:105DE00026010196801791070CF48DCF90E080E09A
:105DF0008ACF2430310509F43FC02530310569F7D9
:105E00000E949C2F892F990F990BB8010E94FA3498
:105E10007ACF019797FD04C0801791070CF473CFD8
:105E2000C801019770CF20912701222339F00196F4
:105E300097FF06C081E080932701D8CF0197F8CF64
:105E4000801791070CF45FCFC801019710922701CA
:105E50005ACF0130110551F22091250130912601D0
:105E6000C9010296801791070CF44DCFC9018095A6
:105E700090958170992747CF8091280190912901B1
:105E80000196B8010E94FA34909329018093280169
:105E9000880F991FFC01EF5CFE4F8081918133CF09
:105EA0008F929F92AF92BF92CF92DF92EF92FF922A
:105EB000CF93DF93EC01688179818A819B816115A1
:105EC00071058105910521F464E279ED8BE597E098
:105ED0002DE133EF41E050E00E947A3049015A0150
:105EE0009B01AC01A7EAB1E40E9499306B017C01EF
:105EF000ACEEB4EFA50194010E94A730DC01CB0108
:105F00008C0D9D1DAE1DBF1DB7FF03C00197A109DC
:105F1000B04888839983AA83BB839F77DF91CF9111
:105F2000FF90EF90DF90CF90BF90AF909F908F90B9
:105F300008950E94502F089581E491E00E94502F0F
:105F40000895B0E0A0E08093410190934201A093B6
:105F50004301B093440108958F929F92AF92BF92F4
:105F6000CF92DF92EF92FF92CF93DF93EC016881A3
:105F700079818A819B81611571058105910521F4E3
:105F800064E279ED8BE597E02DE133EF41E050E0FD
:105F90000E947A3049015A019B01AC01A7EAB1E4A1
:105FA0000E9499306B017C01ACEEB4EFA501940125
:105FB0000E94A730C60ED71EE81EF91EF7FE06C0C7
:105FC00081E0C81AD108E10880E8F80AC882D982BD
:105FD000EA82FB82C701B6019F77DF91CF91FF90E4
:105FE000EF90DF90CF90BF90AF909F908F900895EB
:105FF0008F929F92AF92BF92CF92DF92EF92FF92D9
:10600000609145017091460180914701909148014E
:10601000611571058105910521F464E279ED8BE547
:1060200097E02DE133EF41E050E00E947A304901E2
:106030005A019B01AC01A7EAB1E40E9499306B01BF
:106040007C01ACEEB4EFA50194010E94A730C60E0E
:10605000D71EE81EF91EF7FE06C081E0C81AD10857
:10606000E10880E8F80AC0924501D0924601E0922A
:106070004701F0924801C701B6019F77FF90EF906A
:10608000DF90CF90BF90AF909F908F9008956093D6
:10609000450170934601809347019093480108950C
:1060A000F999FECF92BD81BDF89A992780B50895E0
:1060B000262FF999FECF1FBA92BD81BD20BD0FB624
:1060C000F894FA9AF99A0FBE01960895AA1BBB1B81
:1060D00051E107C0AA1FBB1FA617B70710F0A61BE8
:1060E000B70B881F991F5A95A9F780959095BC0109
:1060F000CD010895052E97FB1EF400940E94913067
:1061000057FD07D00E94AC3007FC03D04EF40C942E
:10611000913050954095309521953F4F4F4F5F4FAF
:10612000089590958095709561957F4F8F4F9F4F03
:1061300008950E94CE30A59F900DB49F900DA49F0E
:10614000800D911D11240895B7FF0C9499300E9481
:106150009930821B930B0895A1E21A2EAA1BBB1B38
:10616000FD010DC0AA1FBB1FEE1FFF1FA217B30723
:10617000E407F50720F0A21BB30BE40BF50B661F39
:10618000771F881F991F1A9469F7609570958095FD
:1061900090959B01AC01BD01CF010895A29FB00174
:1061A000B39FC001A39F700D811D1124911DB29F4B
:1061B000700D811D1124911D08955058BB27AA27E9
:1061C0000E94F5300C94AF320E94A13238F00E9448
:1061D000A83220F039F49F3F19F426F40C949E3233
:1061E0000EF4E095E7FB0C946F32E92F0E94C03269
:1061F00058F3BA17620773078407950720F079F4FC
:10620000A6F50C94FA320EF4E0950B2EBA2FA02DC1
:106210000B01B90190010C01CA01A0011124FF2753
:10622000591B99F0593F50F4503E68F11A16F0404E
:10623000A22F232F342F4427585FF3CF469537954D
:106240002795A795F0405395C9F77EF41F16BA0B12
:10625000620B730B840BBAF09150A1F0FF0FBB1FC0
:10626000661F771F881FC2F70EC0BA0F621F731F09
:10627000841F48F4879577956795B795F7959E3F66
:1062800008F0B0CF9395880F08F09927EE0F9795F7
:10629000879508950E944B3208F481E008950E948A
:1062A00063310C94AF320E94A83258F00E94A132A0
:1062B00040F029F45F3F29F00C946F3251110C9497
:1062C000FB320C949E320E94C03268F39923B1F3E2
:1062D000552391F3951B550BBB27AA27621773070C
:1062E000840738F09F5F5F4F220F331F441FAA1FA0
:1062F000A9F335D00E2E3AF0E0E832D0915050405C
:10630000E695001CCAF72BD0FE2F29D0660F771F09
:10631000881FBB1F261737074807AB07B0E809F0EF
:10632000BB0B802DBF01FF2793585F4F3AF09E3F74
:10633000510578F00C946F320C94FB325F3FE4F31C
:10634000983ED4F3869577956795B795F7959F5FB7
:10635000C9F7880F911D9695879597F90895E1E003
:10636000660F771F881FBB1F621773078407BA0762
:1063700020F0621B730B840BBA0BEE1F88F7E095BD
:1063800008950E94C8316894B1110C94FB320895AD
:106390000E94C83288F09F5798F0B92F9927B751BB
:1063A000B0F0E1F0660F771F881F991F1AF0BA95B9
:1063B000C9F714C0B13091F00E94FA32B1E00895EB
:1063C0000C94FA32672F782F8827B85F39F0B93FDD
:1063D000CCF3869577956795B395D9F73EF490956C
:1063E0008095709561957F4F8F4F9F4F0895E894EA
:1063F00009C097FB3EF490958095709561957F4F0D
:106400008F4F9F4F9923A9F0F92F96E9BB279395BA
:10641000F695879577956795B795F111F8CFFAF4CA
:10642000BB0F11F460FF1BC06F5F7F4F8F4F9F4FFB
:1064300016C0882311F096E911C0772321F09EE859
:10644000872F762F05C0662371F096E8862F70E0BF
:1064500060E02AF09A95660F771F881FDAF7880F99
:106460009695879597F908950E94E23290F09F37AC
:1064700048F4911116F00C94FB3260E070E080E873
:106480009FEB089526F41B16611D711D811D0C9450
:1064900075320C949032990F0008550FAA0BE0E862
:1064A000FEEF16161706E807F907C0F012161306D6
:1064B000E407F50798F0621B730B840B950B39F416
:1064C0000A2661F0232B242B252B21F408950A267C
:1064D00009F4A140A6958FEF811D811D089597F9BC
:1064E0009F6780E870E060E00895882371F4772367
:1064F00021F09850872B762F07C0662311F4992737
:106500000DC09051862B70E060E02AF09A95660FDE
:10651000771F881FDAF7880F9695879597F9089562
:106520009F3F31F0915020F4879577956795B79507
:10653000880F911D9695879597F908959FEF80ECA8
:10654000089500240A9416161706180609060895D9
:1065500000240A9412161306140605060895092E3F
:106560000394000C11F4882352F0BB0F40F4BF2BAE
:1065700011F460FF04C06F5F7F4F8F4F9F4F0895EE
:1065800057FD9058440F551F59F05F3F71F04795E4
:10659000880F97FB991F61F09F3F79F087950895C9
:1065A000121613061406551FF2CF4695F1DF08C0E8
:1065B000161617061806991FF1CF86957105610505
:1065C000089408950E94C832A0F0BEE7B91788F475
:1065D000BB279F3860F41616B11D672F782F8827C8
:1065E000985FF7CF869577956795B11D9395963906
:1065F000C8F30895E894BB2766277727CB0197F95E
:1066000008950E944B3208F48FEF08950E941933C9
:106610000C94AF320E94A13238F00E94A83220F0D0
:10662000952311F00C946F320C949E3211240C942B
:10663000FB320E94C03270F3959FC1F3950F50E07A
:10664000551F629FF001729FBB27F00DB11D639F24
:10665000AA27F00DB11DAA1F649F6627B00DA11DCA
:10666000661F829F2227B00DA11D621F739FB00D70
:10667000A11D621F839FA00D611D221F749F3327E0
:10668000A00D611D231F849F600D211D822F762F79
:106690006A2F11249F5750409AF0F1F088234AF056
:1066A000EE0FFF1FBB1F661F771F881F91505040C2
:1066B000A9F79E3F510580F00C946F320C94FB3289
:1066C0005F3FE4F3983ED4F3869577956795B79549
:1066D000F795E7959F5FC1F7FE2B880F911D969563
:1066E000879597F90895FA01EE0FFF1F309621055F
:1066F0003105A1F16115710561F48038BFE39B0795
:1067000049F168949038810561F08038BFEF9B07AC
:1067100041F099234AF5FF3FE1053105210519F1C3
:10672000E8940894E795D901AA2329F4AB2FBE2F4A
:10673000F85FD0F310C0FF5F70F4A695E0F7F7396B
:1067400050F019F0FF3A38F49F779F930DD00F90D7
:1067500007FC9058089546F00C949E3260E070E07B
:1067600080E89FE308954FE79F775F934F933F93B0
:106770002F930E946E342F913F914F915F910E9411
:1067800006330C94CB3329F416F00C946F320C942E
:10679000FA320C949E320E94C832A8F39638A0F7C1
:1067A00007F80F92E8942BE33AEA48EB5FE70E9480
:1067B0001C330F920F920F924DB75EB70F920E944B
:1067C000B634E8E6F0E00E94FD334F915F91EF911F
:1067D000FF91E595EE1FFF1F49F0FE57E068442743
:1067E000EE0F441FFA95E1F74195550B0E943034A6
:1067F0000F9007FE0C9424340895DF93CF931F93DA
:106800000F93FF92EF92DF927B018C01689406C098
:10681000DA2EEF010E941933FE01E894A59125912B
:10682000359145915591A6F3EF010E94F530FE0197
:106830009701A801DA9469F7DF90EF90FF900F912C
:106840001F91CF91DF9108959B01AC0160E070E052
:1068500080E89FE30C944F310C946F320C9490328B
:106860000E94C832D8F39923C9F3940F511DA3F3A2
:106870009150504094F059F0882332F0660F771F02
:10688000881F91505040C1F79E3F51052CF7880F4B
:10689000911D9695879597F908955F3FACF0983EC6
:1068A0009CF0BB27869577956795B79508F4B160FE
:1068B0009395C1F7BB0F58F711F460FFE8CF6F5FF6
:1068C0007F4F8F4F9F4FE3CF0C94FB3216F00C9409
:1068D00090320C949E3268940C946F320E94C832AD
:1068E000A8F39923C1F3AEF3DF93CF931F930F93D4
:1068F000FF92C92FDD2788232AF02197660F771F83
:10690000881FDAF720E030E040E85FEB9FE388394A
:1069100020F0803E38F021968F770E94DE30E0E94B
:10692000F0E004C00E94DE30EDEBF0E00E94FD33A9
:106930008B01BE01EC01FB2E6F5771097595771F16
:10694000880B990B0E94F93128E132E741E35FE3BC
:106950000E941933AF2D9801AE01FF900F911F9146
:10696000CF91DF910E94F5300C94AF32FA01DC0137
:10697000AA0FBB1F9B01AC01BF5728F42227332766
:106980004427507820C0B75190F4AB2F002446958F
:1069900037952795011CA395D2F3002071F0220FA3
:1069A000331F441FB395DAF30ED00C94DD30613001
:1069B0007105A0E88A07B94630F49B01AC0166274F
:1069C000772788279078309621F02083318342837F
:1069D00053830895DB018F939F930E949930BF9159
:1069E000AF91A29F800D911DA39F900DB29F900D1E
:1069F0001124089597FB072E16F4009407D077FD15
:106A000009D00E94663007FC05D03EF49095819530
:106A10009F4F0895709561957F4F08950E94CE30E5
:106A2000332312F48A1B9B0B0C9418350E94CE3032
:106A3000B7FF0895821B930B0895EE0FFF1F05907B
:106A4000F491E02D09940F931F93CF93DF9382303D
:106A5000910510F482E090E0E091FD04F091FE04D5
:106A600030E020E0B0E0A0E0309799F42115310546
:106A700009F44AC0281B390B24303105D8F58A8126
:106A80009B816115710589F1FB0193838283FE016E
:106A900011C0408151810281138148175907E0F0EC
:106AA0004817590799F4109761F012960C931297B2
:106AB00013961C933296CF01DF91CF911F910F91C6
:106AC00008950093FD041093FE04F4CF21153105C1
:106AD00051F04217530738F0A901DB019A01BD01BB
:106AE000DF01F801C1CFEF01F9CF9093FE0480934D
:106AF000FD04CDCFFE01E20FF31F8193919322504D
:106B0000310939832883D7CF2091FB043091FC04CD
:106B1000232B41F420914B0130914C013093FC0424
:106B20002093FB042091490130914A012115310540
:106B300041F42DB73EB740914D0150914E01241BB9
:106B4000350BE091FB04F091FC04E217F307A0F48D
:106B50002E1B3F0B2817390778F0AC014E5F5F4FB3
:106B60002417350748F04E0F5F1F5093FC044093E5
:106B7000FB04819391939FCFF0E0E0E09CCFCF9313
:106B8000DF930097E9F0FC01329713821282A09103
:106B9000FD04B091FE04ED0130E020E01097A1F477
:106BA00020813181820F931F2091FB043091FC04DE
:106BB0002817390709F061C0F093FC04E093FB0447
:106BC000DF91CF910895EA01CE17DF07E8F54A81FA
:106BD0005B819E0141155105B1F7E901FB83EA8311
:106BE00049915991C40FD51FEC17FD0761F48081BD
:106BF00091810296840F951FE90199838883828190
:106C000093819B838A83F0E0E0E012968D919C91C2
:106C100013970097B9F52D913C911197CD010296EC
:106C2000820F931F2091FB043091FC042817390731
:106C300039F6309751F51092FE041092FD04B0938E
:106C4000FC04A093FB04BCCFD383C2834081518159
:106C5000840F951FC817D90761F44E5F5F4F888175
:106C60009981480F591F518340838A819B81938367
:106C700082832115310509F0B0CFF093FE04E09333
:106C8000FD049ECFFD01DC01C0CF13821282D7CF5D
:0E6C900081E090E0F8940C944D36F894FFCF1C
:106C9E0010273C028B015706570685060118000186
:106CAE000200FFFF0000803F0000803F010000480F
:106CBE004300000800000001000000007800000002
:106CCE00000000010002000300040005000600079A
:106CDE000001000000010000000000FF048000869B
:106CEE000289028D02920200000000800100000065
:106CFE0003000080030000000400001E0000007A64
:106D0E0000000072010000E803000088130000017B
:106D1E0000FFFF0200FFFF03000400FFFF0500FF5E
:106D2E00FF0600070008000000000013070F070011
:106D3E000000000000803F0000A040B002B702BF7C
:106D4E0002C602CF02D702DE02E60200000000A158
:106D5E000458064204EE0473045104650400000056
:106D6E0000DB0F5806351334132009AF0C7D0C14BD
:106D7E000C930BD40B8712950D310D0309B10A221A
:106D8E000BA00A84110C11AD10C717A1082D002AF3
:106D9E00005B005D004446414D205468696E6700FB
:106DAE0076312E3600436F6E66696775726174694F
:106DBE006F6E0053637265656E73617665723A002D
:106DCE00436F6C6F75723A00416C6C6F7720666121
:106DDE0073743A0043616C69627261746500506C41
:106DEE006179204332004F4B2028002900506C61FE
:106DFE0079204334004F4B00446F6E650046616945
:106E0E006C6564005365742073746570733A20006A
:106E1E0042504D3A20004F6E004F666600426C7530
:106E2E00650052656400496E742E004578742E001C
:106E3E00536574200053746570203120736574009F
:106E4E004E6F726D616C00526576657273650042AD
:106E5E006F756E6365004F64642F4576656E0053E3
:106E6E00687566666C650052616E646F6D004356A0
:106E7E00204D6F6465005365742073746570203106
:026E8E00000002
:00000001FF
